:106C96000000050200000301FA0400FA0500030AD9
:106CA6000A5A0B001E0C00FA0D00030E00040F0119
:106CB60064100096120132130AFA14010217010A2F
:106CC6001801FA1905321A010A1B01FA1C05321FAE
:106CD600FFFF20FFFF23011E2400642A00FA2B0079
:106CE600FA2C50782D003D2E004630006432507844
:106CF6003300003432FA3501643601643701503806
:106D06000A643C00643E003C3F000140FFFF411422
:106D160050420A5A430AC84405324500B44600FAAE
:106D26004C00FA500808510596520A32530B465445
:106D36000A96570546590A465A32FA5B010A5C0A10
:106D4600325E000A5F00FE64021C67FFFF6A0A3CAF
:106D56006B00006C32967300017400017801327981
:106D660001327E006481006484FFFF8A00019D0A6F
:106D7600969E00019FFFFFA0013CA2000AA3FFFF11
:106D8600A4FFFFA5FFFFA6FFFFA7FFFFA8FFFFA920
:106D9600FFFF01013C1500022F003C470178480225
:106DA600035601024EFFFF58000261FFFF66000214
:106DB6008500AF8600018700FA89010A990008A1BB
:106DC60000FAFAFAFA01013C1500022F1E3C4701AF
:106DD600784802035601024EFFFF58000261FFFF8A
:106DE6006600028500AF8600018700FA89010A99CC
:106DF6000000A10000FAFAFA01013C1500002F1E5E
:106E06003C47013C4802025601014EFFFF58000074
:106E160061FFFF66000085FFFF86FFFF87FFFF8992
:106E26000102990000A10000FAFAFA0065006F005D
:106E3600790083008D009700A100AC00B600C00069
:106E4600CA00D400DE00E800F200580060006800C6
:106E5600700078008000880090009800A000A800CC
:106E6600B000B800C100C800D000D800DF00E600BE
:106E7600EE00F600410047004D00530059005F0048
:106E860065006C00710077007D00830089008F002B
:106E960095009B00A200A700AC00B200B900C0009C
:0F6EA600C500CA00D200D500DD00E100E700EF13
:10009E0090089AE0900126F090089BE0900095F071
:1000AE0090089CE09000B5F090089DE09000DEF086
:1000BE0090089EE090008AF090089FE09000D0F0AB
:1000CE009008A0E09000EEF09008A1E09000C2F041
:1000DE009008A2E09000E0F09008A3E0900110F0EC
:1000EE009008A4E0900174F09008A5E0900175F0DE
:1000FE009008A6E0900176F0900174E0700C9001EB
:10010E0075E07006900176E060028004C2248002E1
:10011E00D224743690015FF07430900160F0742D2B
:10012E00900161F07432900162F07420900163F0DE
:10013E007438900164F07443900165F07479900105
:10014E0066F0746C900167F07420900168F0742072
:10015E00900169F0742090016AF0742090016BF0A8
:10016E00742090016CF0742090016DF02290089232
:10017E00E0FEA3E0FF7402D39F74019E400C906CCE
:10018E0096120048E493F599804C900061E0D39468
:10019E00054014900892E0FEA3E0FF906C961200CA
:1001AE0048E493F599802F900061E0D394044014B5
:1001BE00900892E0FEA3E0FF906CC9120048E49311
:1001CE00F5998012900892E0FEA3E0FF906CFC126D
:1001DE000048E493F599900892126FD5900892E03A
:1001EE00FEA3E0FFEFB43507EEB40103754D002218
:1001FE0085F97385FA747E017F00E574126FC7E589
:10020E00732FFF50010E8E5A8F5B90001DE0FCA3E2
:10021E00E0FDEF2DFDEE3CFC8C5C8D5D2275A71094
:10022E0085F97385FA747E017F00E574126FC7E558
:10023E00732FFF50010E8E5A8F5B90001DE0FCA3B2
:10024E00E0FDEF2DFDEE3CFC8C5C8D5D22E55DF559
:10025E00FBE55CF5FCD29322E55DF5E9E55CF5EA9C
:10026E00D29422E55DF5EBE55CF5ECD29122E55DED
:10027E00F5EDE55CF5EED29222E55DF5FBE55CF57C
:10028E00FCD28722E55DF5E9E55CF5EAD29022E540
:10029E005DF5EBE55CF5ECE5B54410F5B522E55DF5
:1002AE00F5EDE55CF5EEE5B54420F5B522AE5AAFB9
:1002BE005B74068E048F05FF126FB78C5C8D5DAE7E
:1002CE005AAF5B74068E048F05FF126FE28C5A8D47
:1002DE005BE55B455A60137406C3955BFFE4955A64
:1002EE00FE8E5A8F5B785C12701AE573A85CB800AC
:1002FE0015D3955D4010E573C3955DFFE4955CFEE7
:10030E008E5C8F5D8010E573243CC3955DFFE49594
:10031E005CFE8E5C8F5DAE5CAF5D743B6F4E6006B7
:10032E00743C6F4E701AAE5CAF5D743B6F4E7005D1
:10033E007573018003757302755D3A755C008003F9
:10034E007573002290009CE0B40104C2068002D2B4
:10035E000690009DE0B40104C2078002D20790000F
:10036E00DAE075F0E1A4FFAEF0740A8E048F05FF9B
:10037E00126FB790088AECF0A3EDF074078C068D1F
:10038E0007126FC774038E048F05FF126FB79000AC
:10039E0019ECF0A3EDF07E017F00900098E0126F53
:1003AE00C79000DBE08E048F05FF126FB7740AFF53
:1003BE00126FB78D609000E4E075F0E1A4FFAEF02F
:1003CE00740A8E048F05FF126FB790088EECF0A39F
:1003DE00EDF09000E6E060139000E6E0F5F07416A4
:1003EE0084FF7E00EF9008B6F0800674649008B625
:1003FE00F09000DCE0900078F0900128E090008210
:10040E00F090012AE0FE9000D8E08E0088F0A4FF64
:10041E00AEF0EF9008BEF0900126E090089AF090B2
:10042E0000B5E090089CF09000DEE090089DF09002
:10043E00008AE090089EF0900110E09008A3F090E2
:10044E000174E09008A4F0900175E09008A5F0907A
:10045E000176E09008A6F0A224B34016900174E055
:10046E00700C900175E07006900176E060028002DB
:10047E00C224900174E0B4300F900175E0B44708C7
:10048E00900176E0643B60028004D2258002C22592
:10049E0074E3900077F09000C5E0B40B0874E3901D
:1004AE000077F0805A9000C5E0B419129000DBE09E
:1004BE00906E1C12008CE493900077F080419000B7
:1004CE00C5E0B41E129000DBE0906E3A12008CE490
:1004DE0093900077F080289000C5E0B42812900029
:1004EE00DBE0906E6412008CE493900077F0800F46
:1004FE009000C5E0B446089000BCE0900077F09004
:10050E00007BE0FE9000C2E0B5064B90007DE0FE61
:10051E009000E0E0B5063F90007CE0FE9000EEE03B
:10052E00B5063390007FE0FE900095E0B50627906B
:10053E00007EE0FE9000D0E0B5061B900080E0FE4D
:10054E009000FBE0B5060F900081E0FE9000FCE00D
:10055E006E7003020773900061E0C3940550087437
:10056E0002900111F0801C9000D0E06403600690B0
:10057E0000EEE060087406900111F08006740A9097
:10058E000111F09000D0E0B403089000EEE0640298
:10059E006002800674009000EEF0900095E0B401C9
:1005AE00067400900095F0900095E0B40206740079
:1005BE009000E0F0900095E0B4030674009000ED1A
:1005CE00F09000C2E0601474299000A9F0740090BD
:1005DE0006CEF074009006CFF0800C74009000A947
:1005EE00F074299006CEF09000C2E0B40214742A82
:1005FE009000AAF074009006D2F074009006D3F02A
:10060E00800C74009000AAF0742A9006D2F090002C
:10061E00FBE060147419900115F074009006D6F08A
:10062E0074009006D7F0800C7400900115F07419C8
:10063E009006D6F09000FCE06014741A900116F04B
:10064E0074009006DAF074009006DBF0800C7400F3
:10065E00900116F0741A9006DAF09000E0E0D39450
:10066E00014014741B900113F074009006DEF074B8
:10067E00009006DFF0800C7400900113F0741B9054
:10068E0006DEF09000EEE0B40114741C900114F03C
:10069E0074009006E2F074009006E3F0800C740093
:1006AE00900114F0741C9006E2F09000D0E0B402B9
:1006BE00069000EEE06002801A74059006E6F07473
:1006CE00069006EAF074079006EEF074089006F2B3
:1006DE00F0803074009006E6F074009006E7F07437
:1006EE00009006EAF074009006EBF074009006EEAF
:1006FE00F074009006EFF074009006F2F074009023
:10070E0006F3F0D2239000C2E090007BF09000EE52
:10071E00E090007CF09000E0E090007DF09000D042
:10072E00E090007EF0900095E090007FF09000FB4E
:10073E00E0900080F09000FCE0900081F090009539
:10074E00E090089BF09000D0E090089FF09000EEB3
:10075E00E09008A0F09000C2E09008A1F09000E0B8
:10076E00E09008A2F09000F8E0B401179000297410
:10077E000FF0A374FFF090002BE4F0A3F07402903E
:10078E0000F8F09000F8E0B4034190002BE0FEA3D7
:10079E00E0FF900029E0FCA3E0FD1270127410122D
:1007AE006FC77408120039EF900074F0EF70067482
:1007BE00FF900074F074009000F8F090002AE09022
:1007CE000075F0900029E0900076F0900089E0909E
:1007DE000086F0900088E0900085F09000B7E0C3AE
:1007EE00941E50569000B7E0F404241E900087F03B
:1007FE00900087E075F00684FF7E008F739000876F
:10080E00E075F00684ADF07C008D74900085E0D329
:10081E009574400D900085E0C39574900085F0802E
:10082E000F900085E02406C39574900085F0057343
:10083E00900086E02573900086F0900086E0900090
:10084E004DF090004DE0D3943C400B90004DE0C332
:10085E00943C90004DF090004DE0240F90004EF02F
:10086E0090004DE0241E90004FF090004DE0242D9E
:10087E00900050F090004EE0D3943C400B90004E10
:10088E00E0C3943C90004EF090004FE0D3943C4077
:10089E000B90004FE0C3943C90004FF0900050E05E
:1008AE00D3943C400B900050E0C3943C900050F029
:1008BE00900055E4F090004DE0643B600790004DD1
:1008CE00E0B43C2090004DE0B43B0674029000551D
:1008DE00F090004DE0B43C069000557401F090008D
:1008EE004D7401F0900056E4F090004EE0643B60D1
:1008FE000790004EE0B43C2090004EE0B43B0674EE
:10090E0002900056F090004EE0B43C0690005674F3
:10091E0001F090004E7401F0900057E4F090004FFB
:10092E00E0643B600790004FE0B43C2090004FE045
:10093E00B43B067402900057F090004FE0B43C06B2
:10094E009000577401F090004F7401F0900058E43D
:10095E00F0900050E0643B6007900050E0B43C2003
:10096E00900050E0B43B067402900058F090005096
:10097E00E0B43C069000587401F09000507401F001
:10098E00900089E0FE9000ECE02E90005AF090006E
:10099E005AE0641E600790005AE0B43C0690005A7C
:1009AE00E004F090005AE0641D600790005AE0B435
:1009BE003B0690005AE014F090005AE0D3943C406D
:1009CE000B90005AE0C3943C90005AF090005AE00D
:1009DE00D3941E400D90005AE0C3941E90005BF01D
:1009EE00800A90005AE0241E90005BF075511E9014
:1009FE0000CFE0900051F0900051E075F00F84AF01
:100A0E00F07E00EF4E7006900051E004F090005121
:100A1E00E00475F00F84AFF07E00EF4E700690008C
:100A2E0051E014F0900051E0B47906900051740139
:100A3E00F0900051E0D3943C400F900051E0C394ED
:100A4E003C900051F0D21E8002C21E900051E02454
:100A5E000F900052F0900051E0241E900053F09041
:100A6E000051E0242D900054F0900052E0D3943CBD
:100A7E00400B900052E0C3943C900052F090005313
:100A8E00E0D3943C400B900053E0C3943C90005351
:100A9E00F0900054E0D3943C400B900054E0C3948B
:100AAE003C900054F022C293C294C291C292C2876B
:100ABE00C290E5B554EFF5B5E5B554DFF5B5C29680
:100ACE00C295C2A0C297C2A2C2A1E5B554BFF5B5E8
:100ADE00E5B5547FF5B5E5B554FBF5B5C208755EC1
:100AEE00469000D2E07005756D028003756D03753A
:100AFE00550075540090001074FFF0A374DCF0C222
:100B0E000FC211C213C21574C890003DF074C89084
:100B1E000041F074C8900045F074C8900049F0751B
:100B2E005300755200C203754600E56FB409037594
:100B3E006F0075630090001FE4F0A3F0757010C293
:100B4E000BC20CC20DC20EC2027557007556009034
:100B5E000012E4F0A3F0900014E4F0A3F0C22875A4
:100B6E005900755800900094E075F032A4FFAEF075
:100B7E00900027EEF0A3EFF0900083E4F090008455
:100B8E00E4F0C226D21BC21AD21CC21DC21EC21F44
:100B9E0022755B00755A00AE5AAF5B7402C39F7428
:100BAE00019E5003020C5D906C96120048E49390E7
:100BBE000088126FF80FBF00010EE0FC906C9612C9
:100BCE000048ECFEE493FFEEC39F5026AE5AAF5B97
:100BDE000FBF00010E906C96120048AE5AAF5BE448
:100BEE0093FC906C96120048E493900088126FF874
:100BFE00ECF0AE5AAF5B906C96120048E493900006
:100C0E0088126FF8E0FC906C98120048ECFCE493AC
:100C1E00FDECD39D4019906C98120048E493FC9023
:100C2E006C96120048E493900088126FF8ECF0AEC8
:100C3E005AAF5B74022FFF50010E8E5A8F5B785B9A
:100C4E00740126F6500418E436F64003020BA52272
:100C5E00755B00755A00AE5AAF5B7433BE00039FCE
:100C6E005003020D2B906D98120048E4939000886B
:100C7E00126FF80FBF00010EE0FC906D9812004845
:100C8E00ECFEE493FFEEC39F5026AE5AAF5B0FBF50
:100C9E0000010E906D98120048AE5AAF5BE493FCC3
:100CAE00906D98120048E493900088126FF8ECF063
:100CBE00AE5AAF5B906D98120048E4939000881284
:100CCE006FF8E0FC906D9A120048ECFCE493FDEC9A
:100CDE00D39D4019906D9A120048E493FC906D9844
:100CEE00120048E493900088126FF8ECF0AE5AAF01
:100CFE005B742D6F4E7006755B33755A00AE5AAF2E
:100D0E005B74022FFF50010E8E5A8F5B785B74015D
:100D1E0026F6500418E436F64003020C6422755B86
:100D2E0000755A00AE5AAF5B7433BE00039F50037A
:100D3E00020DF9906DCB120048E493900088126F6B
:100D4E00F80FBF00010EE0FC906DCB120048ECFED8
:100D5E00E493FFEEC39F5026AE5AAF5B0FBF000168
:100D6E000E906DCB120048AE5AAF5BE493FC906DC3
:100D7E00CB120048E493900088126FF8ECF0AE5A54
:100D8E00AF5B906DCB120048E493900088126FF821
:100D9E00E0FC906DCD120048ECFCE493FDECD39D8D
:100DAE004019906DCD120048E493FC906DCB12006B
:100DBE0048E493900088126FF8ECF0AE5AAF5B7473
:100DCE002D6F4E7006755B33755A00AE5AAF5B745D
:100DDE00022FFF50010E8E5A8F5B785B740126F640
:100DEE00500418E436F64003020D3222755B00758E
:100DFE005A00AE5AAF5B7433BE00039F5003020E0F
:100E0E00C7906DFE120048E493900088126FF80FA1
:100E1E00BF00010EE0FC906DFE120048ECFEE49364
:100E2E00FFEEC39F5026AE5AAF5B0FBF00010E9070
:100E3E006DFE120048AE5AAF5BE493FC906DFE124D
:100E4E000048E493900088126FF8ECF0AE5AAF5B56
:100E5E00906DFE120048E493900088126FF8E0FC4B
:100E6E00906E00120048ECFCE493FDECD39D40190B
:100E7E00906E00120048E493FC906DFE120048E460
:100E8E0093900088126FF8ECF0AE5AAF5B742D6F32
:100E9E004E7006755B33755A00AE5AAF5B74022FF7
:100EAE00FF50010E8E5A8F5B785B740126F650044C
:100EBE0018E436F64003020E0022E50C9035F9F8E0
:100ECE00282873020F8E75E700A231B34008E5B5EE
:100EDE004408F5B58006E5B554F7F5B575E710028B
:100EEE000F8E75E700A231B34008E5B54402F5B5A3
:100EFE008006E5B554FDF5B575E710020F8EA231EB
:100F0E0092A2807CA23192A1807675E700A231B3C5
:100F1E004008E5B54440F5B58006E5B554BFF5B5D6
:100F2E0075E710805B75E700A231B34008E5B54464
:100F3E0080F5B58006E5B5547FF5B575E7108040B0
:100F4E00A2319287803AA2319290803475E700A246
:100F5E0031B34008E5B54410F5B58006E5B554EF5C
:100F6E00F5B575E710801975E700A231B34008E5B5
:100F7E00B54420F5B58006E5B554DFF5B575E71037
:1035F900020ED1020ED4020EF0020F0C020F1202BB
:103609000F18020F33020F4E020F54020F5A020F06
:01361900753B
:100F8E002285F97385FA747E017F00E574126FC7AE
:100F9E00E5732FFF50010E8E5A8F5BAC5CAD5DEF8B
:100FAE002DFDEE3CFC8C5C8D5D12025B1202661216
:100FBE00027112027C9000D0E0B4032C75A710854C
:100FCE00F97385FA747E017F00E574126FC7E573BD
:100FDE002FFF50010E8E5A8F5B1202871202921251
:100FEE00029D1202AC75A7002275A71085F97385B4
:100FFE00FA747E017F00E574126FC7E5732FFF5000
:10100E00010E8E5A8F5B7E017F7690010DE0126F7E
:10101E00C7AC5AAD5BED2FFFEC3EFE8E5C8F5DE5EF
:10102E005DF5FDE55CF5FE900078E4F075A70074C3
:10103E001290005DF02285F97385FA747E017F00AF
:10104E00E574126FC7E5732FFF50010E8E5A8F5B3A
:10105E00900019E0FCA3E0FDEF2DFDEE3CFC8C5C56
:10106E008D5DE55DF5FDE55CF5FE220564229000E3
:10107E00D0E0640360079000EEE0B4021EA2D8B385
:10108E004002C293A2D9B34002C294A2DAB3400284
:10109E00C291A2DBB34002C2928044A2D8B3400AEE
:1010AE00C2939000EEE06002C287A2D9B3400AC29A
:1010BE00949000EEE06002C290A2DAB3400EC291AC
:1010CE009000EEE06006E5B554EFF5B5A2DBB34057
:1010DE000EC2929000EEE06006E5B554DFF5B5A2C3
:1010EE00DCB34030A2965006741990005DF0A295C4
:1010FE005006741990005DF0A2A05006741990006D
:10110E005DF0A2975006741990005DF0C296C295DC
:10111E00C2A0C29775D8402285A77275A7109000FD
:10112E00D0E0640360079000EEE0B40224A2D8B3CE
:10113E004002C287A2D9B34002C290A2DAB34006DF
:10114E00E5B554EFF5B5A2DBB34006E5B554DFF5D2
:10115E00B5A2DCB340089000DCE0900078F075D8C2
:10116E00408572A72290F800E4936406600280FE28
:10117E0075B50075840175A70075FFA075EF069013
:10118E000059E4F075C91075A70F75A1C775A700B2
:10119E0075D90075CE0C75A70F75F1FE75F2FF753A
:1011AE00F30775F47875A4BA75A5FF75A60775AE25
:1011BE000075AFFF75D48175D5FF75D6FF75D7FF56
:1011CE0075A70075A20175A14775F80975D8007548
:1011DE00D90475DA0975DB0975DC0975DD0975DE6B
:1011EE000975D84075A71075D80075D90475DA0938
:1011FE0075DB0975DC0975DD0975DE0975D8407575
:10120E00A70075E60875E71075BC0175BE0475BDBF
:10121E006C75BE0775BDA075BE0875BD0175BC00A9
:10122E0075BB1875BC2075BA0875E88075D1137535
:10123E00A70F75E10575E20075C740120AB47597E0
:10124E0000759780740A126FA77597C0E5975420A2
:10125E00700280F8758F0275A700D2AF7598007571
:10126E00A90C75A70F75AB4375ADFB75AC1E75A7B5
:10127E001075C91875CA0075CB0075C80475A7001E
:10128E00758912758E04758C00758A00C2A9D28C70
:10129E00758D00758B00D2ABD28E75B62075D94484
:1012AE00C29974C8F50975080012372275A70FE5A3
:1012BE00FB900067F0E5FA900068F0E5F9900069A0
:1012CE00F075A70090F800E493F5271238419008C6
:1012DE009BE0D39403500790089BE0B40106740082
:1012EE0090089BF074019000D1F090089BE090362E
:1012FE001AF8282873802A802875A70F75F30F75A2
:10130E00A700A2A3400674029000D1F0801375A727
:10131E000F75F31775A700A2A4400674029000D1B2
:01132E00F0CE
:0C361A0002130302130502130702131C25
:10132F009000D1E0B4022AC227123BE07402900071
:10133F00D1F090089BE0903626F828287380108013
:0F134F000E74009000E0F0800674009000EDF046
:0C36260002134C02134E02135002135802
:10135E008028D227123AFF74019000D1F090089B9A
:10136E00E0903632F82828738010800E74009000BA
:0A137E00E0F0800674009000EDF02E
:0C36320002137602137802137A0213824E
:1013880012009E9000DBE07006740A9000DBF0907B
:1013980000BCE0700674E39000BCF09000C2E0046A
:1013A80090007BF0120352E5B54401F5B590F807BB
:1013B800E49390006EF090006EE0440A90006EF0A6
:1013C80090006EE054FE90006EF0740690005FF09E
:1013D8007401900060F090F802E493900061F0745A
:1013E80003900062F07405900063F0741F9000642D
:1013F800F07406900065F0900061E0B4040674048F
:10140800900065F0900061E0B405067405900065F1
:10141800F07407900066F090F804E49390006AF086
:10142800740090006BF090F805E49390006CF090D5
:10143800F806E49390006DF074FF90006FF0120BC3
:101448009F900061E0B40505120D2C801190006199
:10145800E0D394054005120C5E8003120DFA90004B
:10146800F7E0900074F09000AEE0900075F0900006
:10147800AFE0900076F0A2B6B39204A2B3B392059F
:10148800A2A4B39221A2A3B39222900070E4F075B3
:101498006F00743A900788F074FD900789F0900007
:1014A80071E4F0756E0190005DE4F09000D2E0B454
:1014B8000106741A90005DF0C220756300C209D25B
:1014C8000AC202757100C2231236C8755F00756BB7
:1014D800007561007565327566007567007568008E
:1014E800756900756A0090001FE4F0A3F0756C0040
:1014F800D2B2D2A4D2B0D2B1D2A3D2A7D2A6D2A508
:10150800D2B7900094E0D394FA400674FA9000940D
:10151800F07E017F00900076E0126FC7900075E0C2
:101528002FFF50010E900029EEF0A3EFF0EFD394B7
:10153800FFEE940F4007900029E4F0A3F0900074A8
:10154800E0700674FF900074F09000D2E0700575AA
:101558006D028003756D039000D3E0D394014006BB
:1015680074009000D3F09000D9E0C3940A50067438
:101578000A9000D9F09000E3E0700674019000E34F
:10158800F09000E3E0B4FF0674FE9000E3F09000F2
:10159800EAE0D394FE400674FE9000EAF090011051
:1015A800E0D3940240067401900110F0900126E007
:1015B800D3940140067401900126F074019000F064
:1015C800F074019000F1F074009000F8F07400904D
:1015D8000118F0D29C9000C3E0D394044006740430
:1015E8009000C3F09000F5E0D39404400674049092
:1015F80000F5F0E570D3941040037570109006CF95
:10160800E0D3940C400674009006CFF09006D3E027
:10161800D3940C400674009006D3F09006D7E0D31C
:10162800940C400674009006D7F09006DBE0D39443
:101638000C400674009006DBF09006DFE0D3940CB3
:10164800400674009006DFF09006E3E0D3940C4067
:101658000674009006E3F09006E7E0D3940C400689
:1016680074009006E7F09006EBE0D3940C40067403
:10167800009006EBF09006EFE0D3940C400674005F
:101688009006EFF09006F3E0D3940C4006740090B7
:1016980006F3F0D2EC75CF01A298B34005C29812B8
:1016A8003CC1E54D6006A299B3B340028005C299DA
:1016B8001241A2E54E64016005E54EB4040280D5EE
:1016C800C28E7E107F00E564126FC7E58D75F0103D
:1016D800A4FDACF0EF2DFDEE3CFCE58B75F010841D
:1016E800FF7E00ED2FFFEC3EFE8E548F55D28E907C
:1016F80000B5E060099000B5E0C3943D4002805C0D
:10170800900021126FD5900021E0FEA3E0FF900029
:1017180023E0FCA3E0FDEFB50542EEB5043EB217A9
:10172800A203B3401975E700A217B34008E5B54412
:1017380004F5B58006E5B554FBF5B575E7109000DE
:1017480023E0FEA3E0FF900025E0FCA3E0FDEF2DE1
:10175800FDEE3CFC900023ECF0A3EDF09000C2E01D
:1017680060099000C2E0C394034003021801125DAF
:101778006FA203B35009900070E0C3942B4002801D
:10178800069000ACE0F545E54575F002A4FFAEF023
:10179800900890EEF0A3EFF0900099E0C3956140B7
:1017A80007E55FC395605007900890E4F0A3F075D3
:1017B800E700AE2EAF2F900890E0FCA3E0FDEFD33A
:1017C8009DEE9C4015E5B554F7F5B59000C2E0B420
:1017D8000206E5B54402F5B5801C900070E0C3949C
:1017E800415013E5B54408F5B59000C2E0B40206CF
:1017F800E5B554FDF5B575E7109000C2E0B4032ACD
:10180800125E8A75E700AE2EAF2F900890E0FCA319
:10181800E0FDEFD39DEE9C4008E5B554F7F5B580A3
:1018280006E5B54408F5B575E71090009DE0600938
:10183800A2B3300501B3B340028056A2B33005010C
:10184800B3404EA2B3300701B34039A21B403090D9
:101858000082E0D3955E4025900084E070139000EC
:1018680083E0B401069000847401F0900083E004E2
:10187800F0A21AB34005900083E4F0D21AD21BA25A
:1018880007B39205A207B330B301B34004A207928D
:1018980005A2B6300401B35003021F56A2B63004A5
:1018A80001B35003021F56A2B6300601B35003021B
:1018B8001E0B756E009000B5E0B43D1975E700A2E7
:1018C80006B34008E5B554FBF5B58006E5B5440414
:1018D800F5B575E710055EA208B3B35013AE54AF63
:1018E80055900010E0FCA3E0FDEDC39FEC9E400383
:1018F800021AC2E56DB4032EA228B34022E55EB4F5
:101908003B03756D01E55EC3943B500690005D7422
:1019180001F0E55ED3943B4006740290005DF075DB
:101928005E01D2288062E56DB4020A756D01755EAC
:101938003BC21AC21CE55EB43B05755E0180499046
:10194800005DE07034E55EC3943B500690005D7422
:1019580001F0E55ED3943B4006740290005DF0E52B
:101968005EC3943B5002D220E55ED3943B4002D242
:1019780020C296C295C2A0C2979000D2E0B40105D9
:10198800120AB48003755E01AE56AF57AC54AD551C
:10199800EF2DFDEE3CFC74028C068D071200398E8B
:1019A800568F579000B5E060099000B5E0C3943DAC
:1019B80040028049900021E0FEA3E0FF9000B5E0DE
:1019C8008E048F05FF126FB774018C068D07120005
:1019D80039900025EEF0A3EFF0900025E0F8A3E0A1
:1019E800900023C8F0A3C8F0900021E4F0A3F0C24F
:1019F8001775E700E5B554FBF5B575E710A2A4B374
:101A08004002C221A2A3B34002C222A220B34002D4
:101A1800C220B21D900084E0B40111A21AB34004A0
:101A2800D21D8002C21D7402900084F0900084E0F0
:101A3800C394025006A203B3B34002800674029016
:101A48000084F09000DEE0640460079000D0E0B409
:101A5800036290009DE06006900084E07002800DB3
:101A6800A21C301A01B34005900083E4F09000D224
:101A7800E064016006A226B3B3501790009DE060B1
:101A880009A21A301C01B3B3400280067405900005
:101A98005DF0B21CA21BB3401BA21AB34004D21CB7
:101AA8008002C21C9000D2E07006900084E07002B0
:101AB8008002D226C21AC21B803AAE56AF57AC5427
:101AC800AD55EF2DFDEE3CFC74018C068D07120020
:101AD800398E568F57E56DC39402500DAC54AD55F1
:101AE80074B8C39D740B9C40028009120AB4740632
:101AF80090005DF0E55EB43B12740390005DF0D297
:101B0800209000D2E0B40103120AB4AE58AF59AC29
:101B180054AD55EF2DFDEE3CFC8C588D59AE54AFAD
:101B280055EFD39DEE9C4011900017E0FAA3E0FB1F
:101B3800EBC394E8EA940340028006900017126F02
:101B4800D5900014E0FEA3E0FFAC54AD55EF2DFD99
:101B5800EE3CFC900014ECF0A3EDF09000D2E0B461
:101B68000118AE54AF557405126FC77401120039CD
:101B7800900010EEF0A3EFF08011AE54AF55740250
:101B8800126FC7900010EEF0A3EFF0C28E758D00B3
:101B9800758B00756400755501755400D28EE55E2D
:101BA800240E75F00F84AFF07E00EF4E6003021C28
:101BB8003BE56D6013AE56AF57740F126FC79000B8
:101BC80012EEF0A3EFF0800F900014E0F8A3E0907D
:101BD8000012C8F0A3C8F0900012E0FEA3E0FFEFE7
:101BE8004E600B7C7B7D5C126EB58E528F539000DD
:101BF80014E4F0A3F0AE52AF537428BE00039F5014
:101C080010E5632FFF50010E74011200398E528FB8
:101C1800538553639000D9E0A852B8000DD395536B
:101C28004008E55390005CF080099000D9E01490DA
:101C3800005CF09000D0E0B40308900051E0655ECD
:101C48006002800EA21D301E01B34004D21F800224
:101C5800C21FE55E640B6005E55EB429099000C209
:101C6800E06003125A3B90005AE0655E60079000FE
:101C78005BE0B55E03756F00A209B35006A208B316
:101C8800B34003021D3390008EE0B401739001103D
:101C9800E0B40214124343900079E075F0BEA4FF4B
:101CA800AEF08E5C8F5D8056E56775F00A84FF7E26
:101CB80000900588120048E0F55B755A00AE5AAFEF
:101CC8005B9000B3E0126FC774648E048F05FF1237
:101CD8006FB78C5C8D5DE55D900016F0AE5AAF5B1A
:101CE80090008CE0126FC774648E048F05FF126F2A
:101CF800B774BE8C068D07126FC78E5C8F5D801718
:101D080090008CE075F0BEA4FFAEF08E5C8F5D9005
:101D180000B3E0900016F0E561C394CC5006E55D91
:101D2800455C70028003120F8FD209E56DB401067D
:101D3800E55E64116002800C75700190005E7401AC
:101D4800F0756D00E56D6003021E069000D5E06039
:101D58000D900078E0A852B80006955340028048DC
:101D68009000D5E0B4022790004DE0655E601790C2
:101D7800004EE0655E600F90004FE0655E60079082
:101D88000050E0B55E03757003756C00800CC200EE
:101D9800756C0090001FE4F0A3F0900078E06006F6
:101DA800740990005DF0805690004DE0655E601704
:101DB80090004EE0655E600F90004FE0655E600742
:101DC800900050E0B55E3775700190004DE0B55E4B
:101DD8000690005E7401F090004EE0B55E06740255
:101DE80090005EF090004FE0B55E06740390005ED0
:101DF800F0900050E0B55E06740490005EF0A20614
:101E0800B39204A206B330B601B35003021F56754D
:101E18006E019000B5E0B43D1975E700A206B34025
:101E280008E5B54404F5B58006E5B554FBF5B57588
:101E3800E71075E700E5B54401F5B575E710742BB3
:101E4800900070F0A2069204E55ED3944A4014D242
:101E580008E55ED39485400B740490005DF0D220B1
:101E6800755E469000DDE0B40107E56AC39414404E
:101E7800028009120AB4741390005DF0E56AC394F5
:101E8800415009740E90005DF0120AB4900065E0AC
:101E9800FE900061E0C39E4009900061E0D3940881
:101EA800400974FB90005DF0120AB490006AE0608B
:101EB8001590006AE0FE900064E06E600974FE9080
:101EC800005DF0120AB490089BE0600690010DE0F6
:101ED8006002807A74019000D1F090089BE09036FF
:101EE8003EF828287380188016A2A3400674029032
:0F1EF80000D1F0800AA2A4400674029000D1F03D
:0C363E00021EED021EEF021EF1021EFD36
:101F07009000D1E0B40105A227B340028019D2277F
:101F1700120AB4123AFF74019000D1F012009ED257
:101F270023741B90005DF09000D1E0B40206A22755
:101F3700B3B340028019C227120AB4123BE07402FD
:101F47009000D1F012009ED223741B90005DF0A286
:101F570020B34008C296C295C2A0C29790010DE077
:101F6700600CAE52AF537414BE00059F4002803719
:101F7700900095E090364AF8282873802A8028A296
:101F8700A3B35005A222B340028005120FF7D22255
:101F97008015A2A4B35005A221B340028005120FF9
:071FA700F7D2218002800047
:10364A00021F82021F84021F86021F99021FAC02F8
:02365A001FAEA1
:101FAE00A20BB3B35008900051E0655E60030221AE
:101FBE0032A201B35006A200B3B3400302212A900D
:101FCE0000D0E0B4030280030220F1900084E0B45C
:101FDE00020280030220C0A21FB340581201FE90DD
:101FEE000121E0601F90001DE0FEA3E0FF900119AB
:101FFE00E0126FC774C88E048F05FF126FB78C5C2A
:10200E008D5D800A90001DE0F55CA3E0F55DAE5C91
:10201E00AF5D745E126FC774058E048F05FF126F6D
:10202E00B7AE5AAF5BED2FFFEC3EFE8E5C8F5D12AE
:10203E00025B805C12022B900121E0D39404401FBE
:10204E0090001DE0FEA3E0FF90011DE0126FC7742B
:10205E00C88E048F05FF126FB78C5C8D5D800A9061
:10206E00001DE0F55CA3E0F55DAE5CAF5D745E1245
:10207E006FC774058E048F05FF126FB7AE5AAF5B34
:10208E00ED2FFFEC3EFE8E5C8F5D12028775A70072
:10209E009000EEE0B4011975E700A202B34008E526
:1020AE00B54480F5B58006E5B5547FF5B575E710F6
:1020BE00802F1201FE12025B12022B12028775A7ED
:1020CE00009000EEE0B4011975E700A202B34008DB
:1020DE00E5B54480F5B58006E5B5547FF5B575E7F1
:1020EE001080399000EEE0C39402500F1201FE12E0
:1020FE00025BA202B34002D28780211201FE1202BD
:10210E005B12022BAE5AAF5BAC2CAD2DEF2DFDEE5C
:10211E003CFC8C5C8D5D12028775A700C20BD20C45
:10212E00D20DD20EA20CB3B35008900052E0655EF1
:10213E0060030222B9A201B35006A200B3B340035A
:10214E000222B19000D0E0B4030280030222789004
:10215E000084E0B402028003022247A21FB3405B58
:10216E001201FE900121E0D39401401F90001DE06A
:10217E00FEA3E0FF90011AE0126FC774C88E048FA1
:10218E0005FF126FB78C5C8D5D800A90001DE0F527
:10219E005CA3E0F55DAE5CAF5D745E126FC7740557
:1021AE008E048F05FF126FB7AE5AAF5BED2FFFECAB
:1021BE003EFE8E5C8F5D120266805C12022B9001D9
:1021CE0021E0D39405401F90001DE0FEA3E0FF9098
:1021DE00011EE0126FC774C88E048F05FF126FB711
:1021EE008C5C8D5D800A90001DE0F55CA3E0F55DD2
:1021FE00AE5CAF5D745E126FC774058E048F05FF03
:10220E00126FB7AE5AAF5BED2FFFEC3EFE8E5C8FBA
:10221E005D12029275A7009000EEE0B4011975E709
:10222E0000A202B34008E5B54480F5B58006E5B5D9
:10223E00547FF5B575E710802F1201FE120266125B
:10224E00022B12029275A7009000EEE0B4011975F0
:10225E00E700A202B34008E5B54480F5B58006E577
:10226E00B5547FF5B575E71080399000EEE0C39454
:10227E0002500F1201FE120266A202B34002D29069
:10228E0080211201FE12026612022BAE5AAF5BAC17
:10229E002CAD2DEF2DFDEE3CFC8C5C8D5D12029273
:1022AE0075A700D20BC20CD20DD20EA20DB3B35035
:1022BE0008900053E0655E6003022444A201B3500F
:1022CE0006A200B3B3400302243C9000D0E0B40356
:1022DE000280030223FF900084E0B4020280030216
:1022EE0023CEA21FB3405B1201FE900121E0D394D6
:1022FE0003401F90001DE0FEA3E0FF90011BE012C3
:10230E006FC774C88E048F05FF126FB78C5C8D5D1E
:10231E00800A90001DE0F55CA3E0F55DAE5CAF5D5C
:10232E00745E126FC774058E048F05FF126FB7AE01
:10233E005AAF5BED2FFFEC3EFE8E5C8F5D1202718D
:10234E00805C12022B900121E0D39406401F900076
:10235E001DE0FEA3E0FF90011FE0126FC774C88E50
:10236E00048F05FF126FB78C5C8D5D800A90001D87
:10237E00E0F55CA3E0F55DAE5CAF5D745E126FC719
:10238E0074058E048F05FF126FB7AE5AAF5BED2F3B
:10239E00FFEC3EFE8E5C8F5D12029D75A7009000D5
:1023AE00EEE0B4011975E700A202B34008E5B544AA
:1023BE0080F5B58006E5B5547FF5B575E710802F2D
:1023CE001201FE12027112022B12029D75A70090CD
:1023DE0000EEE0B4011975E700A202B34008E5B5BE
:1023EE004480F5B58006E5B5547FF5B575E71080E8
:1023FE003D9000EEE0C3940250131201FE120271E2
:10240E00A202B34006E5B54410F5B580211201FED7
:10241E0012027112022BAE5AAF5BAC2CAD2DEF2D0A
:10242E00FDEE3CFC8C5C8D5D12029D75A700D20BFF
:10243E00D20CC20DD20EA20EB3B35008900054E0CF
:10244E00655E60030225CFA201B35006A200B3B3AE
:10245E0040030225C79000D0E0B40302800302259A
:10246E008A900084E0B402028003022559A21FB3B1
:10247E00405B1201FE900121E0D39403401F9000B7
:10248E001DE0FEA3E0FF90011CE0126FC774C88E22
:10249E00048F05FF126FB78C5C8D5D800A90001D56
:1024AE00E0F55CA3E0F55DAE5CAF5D745E126FC7E8
:1024BE0074058E048F05FF126FB7AE5AAF5BED2F0A
:1024CE00FFEC3EFE8E5C8F5D12027C805C12022B56
:1024DE00900121E0D39407401F90001DE0FEA3E081
:1024EE00FF900120E0126FC774C88E048F05FF1293
:1024FE006FB78C5C8D5D800A90001DE0F55CA3E0EB
:10250E00F55DAE5CAF5D745E126FC774058E048FA1
:10251E0005FF126FB7AE5AAF5BED2FFFEC3EFE8E8E
:10252E005C8F5D1202AC75A7009000EEE0B401194D
:10253E0075E700A202B34008E5B54480F5B5800604
:10254E00E5B5547FF5B575E710802F1201FE120226
:10255E007C12022B1202AC75A7009000EEE0B401C3
:10256E001975E700A202B34008E5B54480F5B580C1
:10257E0006E5B5547FF5B575E710803D9000EEE0A9
:10258E00C3940250131201FE12027CA202B3400643
:10259E00E5B54420F5B580211201FE12027C12022F
:1025AE002BAE5AAF5BAC2CAD2DEF2DFDEE3CFC8C63
:1025BE005C8D5D1202AC75A700D20BD20CD20DC28F
:1025CE000EE57090365CF8282873022BA39000F568
:0125DE00E01C
:06365C000225D80225DB67
:1025DF0090369BF82828731253DD80121253DD803A
:0E25EF000D1254678008125513800312551305
:0F369B000225E60225EB0225F00225F50225FAAD
:1025FD00757002022BA312563F125756125A709045
:10260D000888E0FEA3E0FF740A126FC7900012E085
:10261D00FCA3E0FD74098F02FF126FB78D078C03C9
:10262D008E048A058B06126EB590088CEEF0A3EF22
:10263D00F09000DEE0B40108743CBE00059F40023E
:10264D00800D743C90088CF8E4F0E8A3F0801B90AA
:10265D00088CE0FEA3E0FF74F0BE00039F500B74E6
:10266D00F090088CF8E4F0E8A3F0E53670037536C9
:10267D000190088CE0FEA3E0FFE5362FFF50010E20
:0F268D0090088CEEF0A3EFF075700390005EE004
:033662000226033A
:10269C009036AAF82828738022A230400375700A5D
:1026AC008019A230400375700B8010A23040037566
:0B26BC00700C8007A230400375700D09
:0F36AA000226A30226A50226AE0226B70226C0DC
:1026C700022BA39006CFE060077401F508125B9711
:1026D70090010EE0B4011490010FE0A852B8000475
:1026E70095535007E55FC3956040028009741590C4
:1026F700005DF002277E9000C3E0D39402403F9034
:102707000097E02403A852B800049553500990009D
:1027170099E0D3956150028008D201740890005D5A
:10272700F0900097E0A852B80005D39553500B904E
:102737000099E02403C395615002C20180399000DB
:1027470097E02403A852B8000495535007E55FC3E8
:10275700956040028008D201740890005DF09000F7
:1027670097E0A852B80005D395535009E560240FA8
:10277700C3955F5002C2019000DDE07007E56AC3B0
:10278700941440028002D2019000D2E0B40102D238
:1027970001A2014005757004800A75701090001F32
:0B27A700E4F0A3F0022BA39000C3E0BD
:063665000226CA0227AE96
:1027B2009036B9F828287312442D801212442D80C5
:0E27C2000D1245DB800812468D800312468DF5
:0F36B9000227B90227BE0227C30227C80227CD66
:1027D0009006D3E060077402F508125B97757005E8
:1027E000022BA31247CD7570069006D7E0600774E0
:1027F00003F508125B979006DBE060077404F508A8
:10280000125B97022BA3900016E06006A203B3B3FD
:102810004002801D900016E02529FFAE2850010ED1
:102820008E288F29E55ED3940F5006900016E01491
:10283000F0124A137570079006DFE060077405F523
:1028400008125B979006E3E060077406F508125BD8
:1028500097022BA3900110E0B402031243BB124E67
:10286000437570089006E7E060077407F508125B8F
:10287000979006EBE060077408F508125B97022B4F
:10288000A31251FFA20BB35005A20CB34002800863
:10289000D20BD20CD20DD20E7570109006EFE06004
:1028A000077409F508125B979006F3E06007740A55
:1028B000F508125B97022BA3022BA390003FE0C305
:1028C00094465008C296744690003FF0900055E040
:1028D000B4011DE5362406F53690088CE0FEA3E031
:1028E000FF74062FFF50010E90088CEEF0A3EFF05E
:1028F000900055E0B4021DE536240CF53690088CA6
:10290000E0FEA3E0FF740C2FFF50010E90088CEE48
:10291000F0A3EFF085365B755A0090004DE0F5733B
:102920001202BBE55D90003FF0900008E55AF0A36D
:10293000E55BF0E573900040F0C21090088CE0F584
:102940005AA3E0F55B90004DE0F5731202BBE55D24
:1029500090003DF0900000E55AF0A3E55BF0E573D0
:1029600090003EF0C20F757003022BA3900043E06D
:10297000C3944650139000DEE0B40104C296800276
:10298000C2957446900043F0900056E0B4011DE5F6
:10299000362406F53690088CE0FEA3E0FF74062F7F
:1029A000FF50010E90088CEEF0A3EFF0900056E07F
:1029B000B4021DE536240CF53690088CE0FEA3E049
:1029C000FF740C2FFF50010E90088CEEF0A3EFF077
:1029D00085365B755A0090004EE0F5731202BBE538
:1029E0005D900043F090000AE55AF0A3E55BF0E546
:1029F00073900044F0C21290088CE0F55AA3E0F501
:102A00005B90004EE0F5731202BBE55D900041F073
:102A1000900002E55AF0A3E55BF0E573900042F008
:102A2000C211757003022BA3900047E0C394465077
:102A3000139000DEE0B40104C2968002C2A0744686
:102A4000900047F0900057E0B4011DE5362406F5EC
:102A50003690088CE0FEA3E0FF74062FFF50010EB5
:102A600090088CEEF0A3EFF0900057E0B4021DE563
:102A700036240CF53690088CE0FEA3E0FF740C2F92
:102A8000FF50010E90088CEEF0A3EFF085365B75D9
:102A90005A0090004FE0F5731202BBE55D900047CD
:102AA000F090000CE55AF0A3E55BF0E57390004868
:102AB000F0C21490088CE0F55AA3E0F55B90004F4B
:102AC000E0F5731202BBE55D900045F0900004E56F
:102AD0005AF0A3E55BF0E573900046F0C213757001
:102AE00003022BA390004BE0C3944650139000DEEA
:102AF000E0B40104C2968002C297744690004BF085
:102B0000900058E0B4011DE5362406F53690088C97
:102B1000E0FEA3E0FF74062FFF50010E90088CEE3C
:102B2000F0A3EFF0900058E0B4021DE536240CF558
:102B30003690088CE0FEA3E0FF740C2FFF50010ECE
:102B400090088CEEF0A3EFF085365B755A0090008C
:102B500050E0F5731202BBE55D90004BF090000E63
:102B6000E55AF0A3E55BF0E57390004CF0C21690D7
:102B7000088CE0F55AA3E0F55B900050E0F5731285
:102B800002BBE55D900049F0900006E55AF0A3E530
:102B90005BF0E57390004AF0C21575700380048005
:032BA000028000B0
:10366B000227E30228060228540228810228B80206
:10367B0028BB02296C022A28022AE4022B9F022B68
:04368B00A1022BA3CA
:102BA30090003DE0B55E028003022C45A20F407207
:102BB300900000E0FEA3E0FFEF4E6021AE56AF575A
:102BC300900000E0FCA3E0FD12000374068E048F66
:102BD30005FF126FB7900000ECF0A3EDF090003EFC
:102BE300E0601A900000E0FEA3E0FFAC56AD57EFA3
:102BF3002DFDEE3CFC900000ECF0A3EDF090003EC8
:102C0300E0D39401401A900000E0FEA3E0FFAC562D
:102C1300AD57EF2DFDEE3CFC900000ECF0A3EDF082
:102C2300D20FAE54AF55900000E0FCA3E0FDEFC31C
:102C33009DEE9C400D121044D296C20F74C89000B2
:102C43003DF0A20FB3B3500790003DE0B55E0280A4
:102C53000D121044D29674C890003DF0C20F90003C
:102C63003FE0B55E028003022D00A2104072900087
:102C730008E0FEA3E0FFEF4E6021AE56AF57900091
:102C830008E0FCA3E0FD12000374068E048F05FF29
:102C9300126FB7900008ECF0A3EDF0900040E060F5
:102CA3001A900008E0FEA3E0FFAC56AD57EF2DFDF0
:102CB300EE3CFC900008ECF0A3EDF0900040E0D374
:102CC3009401401A900008E0FEA3E0FFAC56AD5714
:102CD300EF2DFDEE3CFC900008ECF0A3EDF0D210DC
:102CE300AE54AF55900008E0FCA3E0FDEFC39DEEAA
:102CF3009C400AC296744690003FF0C210A210B3E3
:102D0300B3500790003FE0B55E02800AC296744656
:102D130090003FF0C210900041E0B55E02800302D4
:102D23002DC6A2114072900002E0FEA3E0FFEF4E19
:102D33006021AE56AF57900002E0FCA3E0FD120005
:102D43000374068E048F05FF126FB7900002ECF038
:102D5300A3EDF0900042E0601A900002E0FEA3E0D1
:102D6300FFAC56AD57EF2DFDEE3CFC900002ECF0AE
:102D7300A3EDF0900042E0D39401401A900002E0EA
:102D8300FEA3E0FFAC56AD57EF2DFDEE3CFC9000EB
:102D930002ECF0A3EDF0D211AE54AF55900002E077
:102DA300FCA3E0FDEFC39DEE9C401812104490007D
:102DB300DEE0B40104D2968002D295C21174C890A9
:102DC3000041F0A211B3B35007900041E0B55E0299
:102DD30080181210449000DEE0B40104D296800201
:102DE300D29574C8900041F0C211900043E0B55EE3
:102DF300028003022E97A212407290000AE0FEA303
:102E0300E0FFEF4E6021AE56AF5790000AE0FCA3FF
:102E1300E0FD12000374068E048F05FF126FB79056
:102E2300000AECF0A3EDF0900044E0601A90000A71
:102E3300E0FEA3E0FFAC56AD57EF2DFDEE3CFC905A
:102E4300000AECF0A3EDF0900044E0D39401401AA3
:102E530090000AE0FEA3E0FFAC56AD57EF2DFDEE68
:102E63003CFC90000AECF0A3EDF0D212AE54AF5547
:102E730090000AE0FCA3E0FDEFC39DEE9C4015909B
:102E830000DEE0B40104C2968002C295744690004D
:102E930043F0C212A212B3B35007900043E0B55EF1
:102EA3000280159000DEE0B40104C2968002C29550
:102EB3007446900043F0C212900045E0B55E028074
:102EC30003022F68A2134072900004E0FEA3E0FF08
:102ED300EF4E6021AE56AF57900004E0FCA3E0FD37
:102EE30012000374068E048F05FF126FB79000045F
:102EF300ECF0A3EDF0900046E0601A900004E0FED1
:102F0300A3E0FFAC56AD57EF2DFDEE3CFC90000463
:102F1300ECF0A3EDF0900046E0D39401401A90004A
:102F230004E0FEA3E0FFAC56AD57EF2DFDEE3CFCF5
:102F3300900004ECF0A3EDF0D213AE54AF55900023
:102F430004E0FCA3E0FDEFC39DEE9C401812104487
:102F53009000DEE0B40104D2968002D2A0C21374C2
:102F6300C8900045F0A213B3B35007900045E0B5F5
:102F73005E0280181210449000DEE0B40104D29681
:102F83008002D2A074C8900045F0C213900047E0BD
:102F9300B55E028003023039A214407290000CE047
:102FA300FEA3E0FFEF4E6021AE56AF5790000CE05A
:102FB300FCA3E0FD12000374068E048F05FF126F5D
:102FC300B790000CECF0A3EDF0900048E0601A908D
:102FD300000CE0FEA3E0FFAC56AD57EF2DFDEE3C39
:102FE300FC90000CECF0A3EDF0900048E0D39401CA
:102FF300401A90000CE0FEA3E0FFAC56AD57EF2D56
:10300300FDEE3CFC90000CECF0A3EDF0D214AE54BA
:10301300AF5590000CE0FCA3E0FDEFC39DEE9C4098
:10302300159000DEE0B40104C2968002C2A074468B
:10303300900047F0C214A214B3B35007900047E0C6
:10304300B55E0280159000DEE0B40104C2968002F2
:10305300C2A07446900047F0C214900049E0B55EE8
:1030630002800302310AA2154072900006E0FEA31B
:10307300E0FFEF4E6021AE56AF57900006E0FCA391
:10308300E0FD12000374068E048F05FF126FB790E4
:103093000006ECF0A3EDF090004AE0601A90000601
:1030A300E0FEA3E0FFAC56AD57EF2DFDEE3CFC90E8
:1030B3000006ECF0A3EDF090004AE0D39401401A2F
:1030C300900006E0FEA3E0FFAC56AD57EF2DFDEEFA
:1030D3003CFC900006ECF0A3EDF0D215AE54AF55D6
:1030E300900006E0FCA3E0FDEFC39DEE9C401812A8
:1030F30010449000DEE0B40104D2968002D297C25D
:103103001574C8900049F0A215B3B3500790004955
:10311300E0B55E0280181210449000DEE0B40104B2
:10312300D2968002D29774C8900049F0C2159000DD
:103133004BE0B55E0280030231DBA21640729000C1
:103143000EE0FEA3E0FFEF4E6021AE56AF579000B6
:103153000EE0FCA3E0FD12000374068E048F05FF4E
:10316300126FB790000EECF0A3EDF090004CE0600E
:103173001A90000EE0FEA3E0FFAC56AD57EF2DFD15
:10318300EE3CFC90000EECF0A3EDF090004CE0D38D
:103193009401401A90000EE0FEA3E0FFAC56AD5739
:1031A300EF2DFDEE3CFC90000EECF0A3EDF0D216FB
:1031B300AE54AF5590000EE0FCA3E0FDEFC39DEECF
:1031C3009C40159000DEE0B40104C2968002C297D1
:1031D300744690004BF0C216A216B3B3500790008A
:1031E3004BE0B55E0280159000DEE0B40104C296A8
:1031F3008002C297744690004BF0C2169000E0E044
:10320300B402028003023333900072E0D395665018
:1032130064900072E0F4042566FE9000E3E08E0003
:10322300F5F0E884FF7E008F73EFC39410500CEF2A
:103233008573F0A4FDACF08D7380037573FF90006C
:1032430072E0D39573400B900072E0C39573F571F0
:1032530080037571009000FEE0D3957140069000E5
:10326300FEE0F5719000FFE0C3957150069000FFFA
:10327300E0F5718071900072E0C39566FE9000E303
:10328300E08E00F5F0E884FF7E008F73EFC39410A7
:10329300500CEF8573F0A4FDACF08D738003757350
:1032A300FF85735B755A00900072E0255BFFAE5A91
:1032B30050010E8E5A8F5B74FFBE0009D39F4005E9
:1032C300855B7180037571FF9000FEE0D3957140BB
:1032D300069000FEE0F5719000FFE0C39571500683
:1032E3009000FFE0F571A203B3B3500D900073E0BB
:1032F300FE9000EBE0D39E50028014740790005DB3
:10330300F075E700E5B554BFF5B575E71080217595
:10331300A71075E700E5CDC395714008E5B554BF27
:10332300F5B58006E5B54440F5B575E71075A7001A
:103333009000FBE0604E900105E0A852B8000495B0
:10334300535017900104E0A852B8000ED395534090
:1033530009900106E0D395614002801575A710E539
:10336300CDC394BF4004C2A28002D2A275A700803D
:103373001375A710E5CDC394404004C2A28002D2C6
:10338300A275A7009000FCE0604E900108E0A852EF
:10339300B8000495535017900107E0A852B8000EE7
:1033A300D395534009900109E0D3956140028015FC
:1033B30075A710E5CDC394BF4004C2A18002D2A17A
:1033C30075A700801375A710E5CDC394404004C2D0
:1033D300A18002D2A175A700E56FC39409500AA288
:1033E300EDB34005C2ED126031AE54AF557410C356
:1033F3009F74279E400C900071E0C3945A400302CF
:1034030035F6A208B34009120AB4740690005DF0C1
:10341300A20AB3500EE561D394334007E561C39428
:10342300CC40028041900110E0B402141243439057
:103433000079E075F050A4FFAEF08E5C8F5D800FD5
:1034430090008CE075F050A4FFAEF08E5C8F5DE5CC
:103453005D455C6011E5B54401F5B5742B900070D2
:10346300F0120F8FD20A900071E0D394014007E568
:1034730061C3941A40028002C20A9006CFE060073B
:103483007401F508125B979006D3E060077402F5A8
:1034930008125B979006D7E060077403F508125B88
:1034A300979006DBE060077404F508125B979006BB
:1034B300DFE060077405F508125B979006E3E060B0
:1034C300077406F508125B979006E7E06007740738
:1034D300F508125B979006EBE060077408F5081295
:1034E3005B979006EFE060077409F508125B97900D
:1034F30006F3E06007740AF508125B97900071E029
:10350300C3945A5010E56FB40909900071E004F0B8
:10351300756F00803BE56FB40903756F0075550047
:10352300755400758D00758B00756400900070E014
:10353300C394415008900070E004F08006744190F9
:103543000070F0900070E0B44106E5B554FEF5B5A7
:10355300900071E0D394014007E56AC394414002AF
:103563008009740E90005DF0120AB490089BE0602D
:103573000690010DE06002807A74019000D1F09012
:10358300089BE090368FF828287380188016A2A332
:10359300400674029000D1F0800AA2A4400674028F
:0435A3009000D1F0D3
:0C368F0002358D02358F02359102359D09
:1035A7009000D1E0B40105A227B340028019D227C9
:1035B700120AB4123AFF74019000D1F012009ED2A1
:1035C70023741B90005DF09000D1E0B40206A2279F
:1035D700B3B340028019C227120AB4123BE0740247
:1035E7009000D1F012009ED223741B90005DF00270
:0235F700169D1F
:10693A000000010001400160018001A001C001E0E6
:10694A0002000300039603B603D603F4040005000D
:10695A000512052405360548055A056C057E05907D
:10696A0005A805C005DE0600061406280646066EBA
:10697A0006AE05CF00FF013F015F017F019F01BF06
:10698A0001DF01FF02FF039503B503D503F303FFFC
:10699A0004FF05110523053505470559056B057DD6
:1069AA00058F05A705BF05CE05F10613062706457F
:1069BA00066D06AD06ED05DD0FAA0FA50F9F0F9A0E
:1069CA000F940F8D0F870F800F780F710F680F606C
:1069DA000F570F4E0F450F3B0F300F250F1A0F0E93
:1069EA000F020EF50EE80EDB0ECC0EBE0EAE0E9F9B
:1069FA000E8E0E7D0E6C0E5A0E470E340E200E0CA5
:106A0A000DF70DE20DCB0DB50D9D0D850D6D0D54D8
:106A1A000D3A0D200D050CE90CCE0CB10C940C7638
:106A2A000C580C3A0C1B0BFB0BDB0BBB0B9A0B79B0
:106A3A000B570B350B130AF10ACE0AAB0A870A6405
:106A4A000A400A1C09F809D409B0098C09670943E4
:106A5A00091F08FB08D608B2088E086A08460823E8
:106A6A0007FF07DC07B9079607730751072F070DBA
:106A7A0006EC06CA06AA068906690649062A060A0D
:106A8A0005EC05CD05B0059205750558053C0520B0
:106A9A00050504EA04CF04B5049C04820469045180
:106AAA0004390422040B03F403DE03C803B2039D72
:106ABA00038903750361034D033B0328031603048B
:106ACA0002F202E102D102C002B002A002910282E5
:106ADA000273026502570249023C022F0222021681
:106AEA00020901FD01F201E601DB01D001C601BB89
:106AFA0001B101A7019D0194018B01820179017005
:106B0A00016801600158015001480141013901320F
:106B1A00012B0125011E01180111010B010500FFBE
:106B2A0000FA0FA60FA00F990F920F8B0F840F7CFC
:106B3A000F740F6B0F620F580F4E0F430F380F2C45
:106B4A000F1F0F120F050EF70EE80ED80EC80EB75C
:106B5A000EA50E930E800E6C0E580E420E2C0E15BC
:106B6A000DFD0DE40DCB0DB10D950D790D5D0D3FAC
:106B7A000D200D010CE10CC00C9E0C7C0C590C353F
:106B8A000C100BEA0BC40B9E0B760B4F0B260AFD5F
:106B9A000AD40AAA0A800A550A2A09FF09D409A8A6
:106BAA00097C0950092508F908CD08A10875084A81
:106BBA00081E07F307C8079D07730749072006F74A
:106BCA0006CE06A6067E06570630060A05E405BF67
:106BDA00059B057705540532051004EF04CE04AE73
:106BEA00048F047104530435041903FD03E203C737
:106BFA0003AD0394037B0363034B0334031E0308AF
:106C0A0002F302DE02CA02B602A30291027F026DF9
:106C1A00025C024C023C022C021D020E020001F22E
:106C2A0001E401D701CA01BE01B101A6019A018F8F
:106C3A000185017A01700166015D0153014A014132
:106C4A00013901310129012101190112010B010444
:106C5A0000FD00F700F000EA00E400DE00D900D3EE
:106C6A0000CE00C900C400BF00BA00B500B100AD33
:106C7A0000A800A400A0009C009900950091008E35
:0C6C8A00008A008700840081007E007BEF
:1036C800754700900892E4F0A3F07531007530005A
:1036D800754D00754E00C22BD22D90089BE06002FC
:1036E800D22374FE900894F8E4F0E8A3F074FE90F6
:1036F8000898F8E4F0E8A3F074FE900896F8E4F06F
:10370800E8A3F0745A9008BAF0745A9008BBF0D243
:103718002EC229C230C22FC22A22750B00750A0098
:10372800AE0AAF0BAC08AD09EDC39FEC9E40167412
:10373800FF126FA775CF01780B740126F650041895
:10374800E436F650DB22C2AF75D904758F0375B71E
:10375800A575B7F190F800E4F0758F0175B7A575F8
:10376800B7F1E52790F800F075B7A575B7F190F8AF
:1037780001E4F075B7A575B7F19008AEE090F802CE
:10378800F075B7A575B7F19008B2E090F803F07539
:10379800B7A575B7F19008AFE090F804F075B7A534
:1037A80075B7F19008B0E090F805F075B7A575B752
:1037B800F19008B1E090F806F075B7A575B7F190EB
:1037C80008B3E090F807F0758F0075D944D2AF229E
:1037D800900059E0B4AB61C2AF75D90475B62275D3
:1037E800F522758F0375B7A575B7F1740090F600CB
:1037F800F0758F01755B00755A00AE5AAF5B741394
:10380800BE00279F402475B7A575B7F190089A1296
:103818000048E0FC90F600120048ECF0785B740178
:1038280026F6500418E436F650D0758F0075F51159
:1038380075B62075D944D2AF22C2AF75F52275D9B5
:1038480004755B00755A00AE5AAF5B7413BE002254
:103858009F401F90F600120048E493FC90089A12CB
:103868000048ECF0785B740126F6500418E436F64C
:1038780050D575D94475F511D2AF22900059E0B4EE
:10388800AA0280030239C0C2AF75D90475B6227581
:10389800F522758F0375B7A575B7F1740090EE0022
:1038A800F075B7A575B7F1740090F000F075B7A57D
:1038B80075B7F1740090F200F075B7A575B7F1749B
:1038C8000090F400F0758F01755B00755A00AE5AD0
:1038D800AF5B74FFC39F74019E402475B7A575B78D
:1038E800F1900088120048E0FC90EE00120048ECCD
:1038F800F0785B740126F6500418E436F650CF755C
:103908005B00755A00AE5AAF5B74FFC39F74019E8B
:10391800402475B7A575B7F1900288120048E0FCFD
:1039280090F000120048ECF0785B740126F6500421
:1039380018E436F650CF755B00755A00AE5AAF5B87
:1039480074FFC39F74019E402475B7A575B7F190A5
:103958000488120048E0FC90F200120048ECF0786D
:103968005B740126F6500418E436F650CF755B00F8
:10397800755A00AE5AAF5B74FFC39F74019E402412
:1039880075B7A575B7F1900688120048E0FC90F469
:1039980000120048ECF0785B740126F6500418E435
:1039A80036F650CF758F0075F51175B62075D94468
:1039B800D2AF743A900788F022900059E0B4AA0276
:1039C8008003023AFEC2AF75D90475B62275F52296
:1039D800758F0375B7A575B7F1740090E600F0759B
:1039E800B7A575B7F1740090E800F075B7A575B77D
:1039F800F1740090EA00F075B7A575B7F1740090FE
:103A0800EC00F0758F01755B00755A00AE5AAF5B1C
:103A180074FFC39F74019E402475B7A575B7F190D4
:103A28000088120048E0FC90E600120048ECF078AC
:103A38005B740126F6500418E436F650CF755B0027
:103A4800755A00AE5AAF5B74FFC39F74019E402441
:103A580075B7A575B7F1900288120048E0FC90E8A8
:103A680000120048ECF0785B740126F6500418E464
:103A780036F650CF755B00755A00AE5AAF5B74FFCF
:103A8800C39F74019E402475B7A575B7F19004884B
:103A9800120048E0FC90EA00120048ECF0785B74F1
:103AA8000126F6500418E436F650CF755B00755AB7
:103AB80000AE5AAF5B74FFC39F74019E402475B774
:103AC800A575B7F1900688120048E0FC90EC00124A
:103AD8000048ECF0785B740126F6500418E436F6DA
:103AE80050CF758F0075F51175B62075D944D2AFD2
:103AF800743A900788F022C2AF75D90475F522751B
:103B08005B00755A00AE5AAF5B74FFC39F74019E89
:103B1800401F90EE00120048E493FC9000881200C9
:103B280048ECF0785B740126F6500418E436F65039
:103B3800D4755B00755A00AE5AAF5B74FFC39F74AF
:103B4800019E401F90F000120048E493FC90028808
:103B5800120048ECF0785B740126F6500418E4363D
:103B6800F650D4755B00755A00AE5AAF5B74FFC34C
:103B78009F74019E401F90F200120048E493FC904D
:103B88000488120048ECF0785B740126F65004189B
:103B9800E436F650D4755B00755A00AE5AAF5B74C4
:103BA800FFC39F74019E401F90F400120048E493E5
:103BB800FC900688120048ECF0785B740126F650F9
:103BC8000418E436F650D475F51175D944D2AF749B
:103BD8003A900788F0C22C22C2AF75D90475F52235
:103BE800755B00755A00AE5AAF5B74FFC39F7401D2
:103BF8009E401F90E600120048E493FC9000881253
:103C08000048ECF0785B740126F6500418E436F6A8
:103C180050D4755B00755A00AE5AAF5B74FFC39FF2
:103C280074019E401F90E800120048E493FC900243
:103C380088120048ECF0785B740126F6500418E40A
:103C480036F650D4755B00755A00AE5AAF5B74FFF8
:103C5800C39F74019E401F90EA00120048E493FC41
:103C6800900488120048ECF0785B740126F6500442
:103C780018E436F650D4755B00755A00AE5AAF5B3F
:103C880074FFC39F74019E401F90EC00120048E42B
:103C980093FC900688120048ECF0785B740126F6D5
:103CA800500418E436F650D475F51175D944D2AFDE
:103CB800743A900788F0D22C22E54E64046006E539
:103CC8009964FF60028031A22B4004D22B8027E543
:103CD8004E600874E6254E90005DF0E54D6008746E
:103CE800F0254D90005DF0E54EB4010280FE754E62
:103CF80000754D00C22B8002C22BE54E9068AAF8D1
:103D0800282873754E00E599B4FF03754D01E599B0
:103D1800B4FE03754D02E599B4FD03754D03E599AD
:103D2800B4FC03754D04E599B4FA03754D05E5999E
:103D3800B4FB06754E01120AB4E599B4F906754E3E
:103D480004120AB4E599D394E54007E599C394F0C1
:103D58004002801685994F754E027E017F00E54F1F
:103D6800C394E6126FC78E328F33900892E4F0A3A3
:103D7800F0E599D394C44007E599C394E6400280DE
:103D88002885994F754E0374E5C3954FF533753201
:103D980000AE32AF3390693A126F96E493F874012B
:103DA80093900892C8F0A3C8F0D2990241A1900854
:103DB8009AE0700AA224B35005A225B340028042BB
:103DC800900892E0FEA3E0FF74FFBE00039F500935
:103DD800EFC39446EE94064011900892E0FEA3E0EB
:103DE800FFEFD3946DEE94064013900892E0FEA383
:103DF800E0FF900088120048E599F08003859974E7
:103E08008011900892E0FEA3E0FF9000881200481D
:103E1800E599F0900892126FD5900892E0FEA3E021
:103E2800FFEFB40106EEB407028003023F9A900741
:103E380088E0B43C028003023F9AA224B35005A252
:103E480025B34003023F11C29C90089AE0900126D6
:103E5800F090089BE0900095F090089CE09000B5E9
:103E6800F090089DE09000DEF090089EE090008AB7
:103E7800F090089FE09000D0F09008A0E09000EE4D
:103E8800F09008A1E09000C2F09008A2E09000E055
:103E9800F09008A3E0900110F09008A4E09001745D
:103EA800F09008A5E0900175F09008A6E0900176E2
:103EB800F0120352900074E09000F7F0900075E063
:103EC8009000AEF0900076E09000AFF074AB9000F8
:103ED80059F01237D874AA900059F0A22CB34005B3
:103EE8001239C18003123883900059E4F0900174AC
:103EF800E0700C900175E07006900176E060028039
:103F080004C2248002D224807EC29C900126E090C4
:103F1800089AF0900095E090089BF09000B5E0902A
:103F2800089CF09000DEE090089DF090008AE090F8
:103F3800089EF09000D0E090089FF09000EEE0908E
:103F480008A0F09000C2E09008A1F09000E0E09096
:103F580008A2F0900110E09008A3F074009008A463
:103F6800F074009008A5F074009008A6F074AB9067
:103F78000059F01237D874AA900059F012388312F9
:103F880039C17599FB80FED29C754E00754D007540
:103F980099FB0241A1900892E0FEA3E0FFEF4E706A
:103FA80006859931753000900892E0FEA3E0FF7411
:103FB800016F4E701BAC30AD31AA32AB33ED2BFB29
:103FC800EC3AFA8A068B07900088120048E599F0C7
:103FD800900892126FD5900892E0FEA3E0FF740259
:103FE8006F4E7021AC30AD3174566D4C7006E54F94
:103FF80064E660028003120AB4120352854F997571
:104008004E00754D000241A1900892E0FEA3E0FF2A
:10401800900088120048E599F0900892126FD590A8
:104028000892E0FEA3E0FFAC32AD338F028E038C22
:10403800068D0790697E126F96E493F9740193FEDA
:10404800EAD39EEB994009854F99754E00754D004E
:104058000241A1900892E0FEA3E0FF9000881200C0
:1040680048E599F0900892126FD5900892E0FEA367
:10407800E0FFEFB40006EEB4010280030241A19014
:104088000069E0D394C7400B900069E0C394C8F579
:1040980050801A900069E0D39463400B900069E067
:1040A800C39464F5508006900069E0F550E55075BA
:1040B800F002A4FFAEF08F73EF900088126FF8EF54
:1040C800FCE0FDEC90008B126FF8EDFCE0FDEC2DB0
:1040D800B5500280030241920FEF900088126FF8EA
:1040E800E573FFE0FCEF90008C126FF8ECFFE0FC4A
:1040F800EFC39CB550028003024192E57390008A99
:10410800126FF8E573FFE0FCEF90008D126FF8EC8A
:10411800FFE0FCEF2CB55072E57390008E126FF83B
:10412800E0C395509008AEF0E57390008F126FF8D9
:10413800E0C395509008AFF0E573900092126FF8C5
:10414800E0C395509008B0F0E573900093126FF8B3
:10415800E0C395509008B1F0E573900094126FF8A1
:10416800E0C395509008B2F0E573900095126FF88F
:10417800E0C395509008B3F012374E7599F97464FE
:10418800F50975080012372280FE7599FF7464F5E9
:094198000975080012372280FEAF
:0F68AA00023D0B023DB6023F9D02401002405BD3
:1041A10022E54D9068B9F82828730242869008925A
:1041B100E0FEA3E0FF90005F120048E0F59990084F
:1041C10092126FD5900892E0FEA3E0FF74116F4E3A
:1041D1007003754D00024286856E990242869008F1
:1041E10092E0FEA3E0FF900088120048E0F599EF0D
:1041F100B40107EEB40703754D00900892126FD514
:07420100024286900893E0E1
:0F68B9000241AB0241AE0241D90241DF0242046B
:1042080090690DF82828738553998067855F998090
:1042180062856199805D8565998058856799805325
:10422800856899804E8569998049856A9980449006
:104238000020E0F599803CA22DB340077599FAC299
:104248002D8017A223B3400575990F800B90005D50
:10425800E0F59990005DE4F0C2238017856B9980A2
:1042680012856699800D856C9980087599FC800384
:03427800754D0081
:10690D0002420F02421402421902421E02422302A7
:10691D00422802422D02423202423702423F0242D7
:0D692D006402426902426E02427302427827
:0B427B00900892126FD5800312017BA7
:0368C80002428306
:1042860022E537255BFFAE5A50010E9000881200DA
:1042960048E0F538E537255BFFAE5A50010E0FBFF3
:1042A60000010E900088120048E0F539853F3BE595
:1042B60038B539058538378041E539D39538401DFD
:1042C600E539C39538853AF0A4FFAEF0E53B8E0498
:1042D6008F05FF126FB7ED2538F537801DE538C31A
:1042E6009539853AF0A4FFAEF0E53B8E048F05FFC5
:1042F600126FB7EDF4042538F53722E539D3953832
:10430600401DE539C39538853AF0A4FFAEF0E53B8C
:104316008E048F05FF126FB7ED2538F537801DE542
:1043260038C39539853AF0A4FFAEF0E53B8E048F8D
:1043360005FF126FB7EDF4042538F5372290008E8D
:10434600E0B40170E56775F00A84FF7E008F37E5FB
:104356006775F00A84ADF07C008D3A753F0A755A90
:1043660005755B24E537C394115005124287800614
:104376009005BDE0F537E537900079F0E56775F013
:104386000A84FF7E008F37E56775F00A84ADF07CFE
:10439600008D3A753F0A755A05755B5AE537C39421
:1043A60011500512428780069005F3E0F537E53790
:1043B600900016F02290008EE0B4016AE56775F071
:1043C6000A84FF7E008F37E56775F00A84ADF07CBE
:1043D600008D3A753F0A755A05755B36E537C39405
:1043E60011500512428780069005CFE0F5378537D4
:1043F6004BE56775F00A84FF7E008F37E56775F039
:104406000A84ADF07C008D3A753F0A755A05755BD6
:1044160048E537C39411500512428780069005E19E
:10442600E0F53785374C22E55F75F00484FF7E00A2
:104436008F37E55F75F00484ADF07C008D3A753FEB
:1044460004755A01755B00E537C3943F5005124267
:104456008780069001C7E0F53785372975280090D3
:10446600005CE075F020A4FFAEF09000D9E08E0469
:104476008F05FF126FB78D379000C1E0D3955F505F
:10448600030245339000E5E0D3955F4010ED9001BF
:10449600C8126FF8E0F52B752A000245309000B07F
:1044A600E0D3955F4043E5379001C8126FF8E0F519
:1044B60038E5379001E8126FF8E0F5399000E5E04D
:1044C600F404255FF53A9000B0E0FE9000E5E0F4D4
:1044D600042EF53BE538B539058538378003124398
:1044E6000185372B752A008041E5379001E8126F68
:1044F600F8E0F538E537900208126FF8E0F53990E4
:1045060000B0E0F404255FF53A9000C1E0FE9000AB
:10451600B0E0F4042EF53BE538B53905853837802B
:104526000312430185372B752A000245DA9000E80D
:10453600E0D3955F5011E537900248126FF8E0F529
:104546002B752A000245DA9000B1E0D3955F5043FF
:10455600E537900228126FF8E0F538E53790024803
:10456600126FF8E0F5399000B1E0F404255FF53AF2
:104576009000E8E0FE9000B1E0F4042EF53BE5384B
:10458600B53905853837800312430185372B752ADF
:10459600008041E537900208126FF8E0F538E537FC
:1045A600900228126FF8E0F5399000C1E0F4042576
:1045B6005FF53A9000B1E0FE9000C1E0F4042EF5FC
:1045C6003BE538B539058538378003124301853711
:1045D6002B752A00229000F9E0F53C753F11755ABB
:1045E60002755B00AE52AF53E53C75F00FA4FDAC0F
:1045F600F0EDD39FEC9E4021E53C8E048F05FF1223
:104606006FB7ED75F010A4FFAEF0E55F75F011849D
:10461600FD7C00ED2FF53D800EE55F75F01184FF02
:104626007E00EF24F0F53D853D37E55F75F011849A
:10463600AFF07E008F3A12428785373EAE52AF53B7
:104646009000F9E075F00FA4FDACF0EDD39FEC9E61
:104656004028755A02755B10853D37124287853EA4
:1046660038853739AE52AF53E53C8E048F05FF12BD
:104676006FE28D3A853C3B12430185372975280048
:10468600752B64752A00229000F9E0F53C753F1100
:10469600755A02755B00AE52AF53E53C75F00FA438
:1046A600FDACF0EDD39FEC9E4021E53C8E048F05DA
:1046B600FF126FB7ED75F010A4FFAEF0E56175F06F
:1046C6001184FD7C00ED2FF53D800EE56175F0113E
:1046D60084FF7E00EF24F0F53D853D37E56175F0FA
:1046E6001184AFF07E008F3A12428785373EAE5274
:1046F600AF539000F9E075F00FA4FDACF0EDD39F39
:10470600EC9E4028755A02755B10853D371242872C
:10471600853E38853739AE52AF53E53C8E048F055A
:10472600FF126FE28D3A853C3B12430185372975AE
:104736002800E56B6017E56BC394FE50109000ED02
:10474600E0B402099000DBE0D3940B50028017AE70
:1047560028AF29E56B126FC774E78E048F05FF1229
:104766006FB78C288D299000C3E0B40453E55F75BC
:10477600F00484FF7E008F37E55F75F00484ADF0AA
:104786007C008D3A753F04755A01755B00E537C3A9
:10479600943F500512428780069001C7E0F537AE78
:1047A60028AF29E537126FC774648E048F05FF1290
:1047B6006FB7AE28AF29EF2DFDEE3CFC8C288D2976
:1047C600752B64752A002290008EE0B40146E567D9
:1047D60075F00A84FF7E008F37E56775F00A84ADB1
:1047E600F07C008D3A753F0A755A05755B00E53712
:1047F600C3941150051242878006900599E0F5375B
:10480600AE2AAF2BE5372FFF50010E746412700AE3
:104816008E2A8F2B90008FE0B40146E56875F00A6A
:1048260084FF7E008F37E56875F00A84ADF07C0062
:104836008D3A753F0A755A05755B6CE537C3941159
:1048460050051242878006900605E0F537AE2AAF7E
:104856002BE5372FFF50010E746412700A8E2A8FD3
:104866002B90009EE0B40249E56AC3944175F005B9
:1048760084FF7E008F37E56A75F00584ADF07C0015
:104886008D3A753F05755A06755B00E537C3941377
:104896005005124287800690069BE0F537AE2AAF98
:1048A6002BE5372FFF50010E746412700A8E2A8F83
:1048B6002B9000E0E0B40202800302496CE55F75CC
:1048C600F01584FF7E008F37E55F75F01584ADF037
:1048D6007C008D3A753F15755A03755BF4E537C351
:1048E600940B50051242878006900487E0F537E561
:1048F6003775F0FFA4FFAEF09000E1E08E048F055F
:10490600FF126FB7ED900072F0E56675F078A4FFC0
:10491600AEF074FF8E048F05FF126FB78C5A8D5B55
:1049260074028C068D071200398F37AC5AAD5B7452
:1049360004FF126FE28D3A753F04755A06755B28BF
:10494600E537C3941D500512428780069006CDE0D8
:10495600F537AE2AAF2BE5372FFF50010E746412E0
:10496600700A8E2A8F2B90008DE0B4025DE561758A
:10497600F064A4FFAEF074081200398E5C8F5D748B
:10498600058E048F05FF126FB78D37AE5CAF5D7471
:10499600058E048F05FF126FE28D3A753F05755A35
:1049A60005755BDEE537C394135005124287800612
:1049B600900679E0F537AE2AAF2BE5372FFF500189
:1049C6000E746412700A8E2A8F2B9000CFE0703C12
:1049D60090005CE075F00584FF7E008F3790005CE8
:1049E600E075F00584ADF07C008D3A753F05755A8B
:1049F60005755BC0E537C3941D50051242878006D6
:104A0600900665E0F537E53790007AF0229000963B
:104A1600E0B401179008B5E0252BFFAE2A50010E31
:104A26009000EAE012700A8E2A8F2B90010EE0B4F5
:104A3600011490010FE0A852B8000495535007E501
:104A46005FC39560400280139000B8E0252BFFAE4F
:104A56002A50010E8E2A8F2B024E42900096E0B409
:104A66000306A229B3B3400280509008BEE070103E
:104A76009008B8E0C39405A852B8000695534002C2
:104A860080109000B8E0252BFFAE2A50010E8E2A2A
:104A96008F2B9008BEE0600D9008B8E0A852B800D1
:104AA600069553400280109000B8E0252BFFAE2AF1
:104AB60050010E8E2A8F2B024E42900090E0B402D7
:104AC600028003024E42900093E0602FE567D39484
:104AD600464028900017E0FEA3E0FF9000CEE07568
:104AE600F003A4FDACF0EFD39DEE9C400E9000F2D7
:104AF600E0A852B80005D395535003024E429000E9
:104B0600C3E0B403028003024CA685615B755A00BC
:104B160090009AE0A852B800049553500E90009B5E
:104B2600E0A85AB80005D3955B5003024CA3E56193
:104B360075F002A4FFAEF074158E048F05FF126F98
:104B4600B78C068D07900618120048FEE0FFEE901F
:104B56000092E0FEEF8E0088F0A4FFAEF074648E43
:104B6600048F05FF126FB78C5A8D5B90005CE07561
:104B7600F018A4FFAEF09000D9E08E048F05FF1266
:104B86006FB78C068D07900630120048AE5AAF5BA1
:104B9600E0126FC774648E048F05FF126FB78C5ACC
:104BA6008D5BE565A85AB80077D3955B4072E565DD
:104BB600C3955BFFE4955AFE8E5A8F5B7428BE0040
:104BC600039F500C755B28755A00740D90005DF0BC
:104BD600AE5AAF5B900093E0126FC774288E048FB5
:104BE60005FF126FB78C5A8D5BAE28AF29740A8EFB
:104BF600048F05FF126FB78D068C07AC5AAD5BCFDD
:104C0600CECF120003740A8E048F05FF126FB78C85
:104C16005A8D5BAE28AF291270128E288F29807D9F
:104C2600E565A85AB80004955B5072AE5AAF5BE5CD
:104C36006512700A8E5A8F5B7428BE00039F500C53
:104C4600755B28755A00740D90005DF0AE5AAF5B27
:104C5600900093E0126FC774288E048F05FF126FC1
:104C6600B78C5A8D5BAE28AF29740A8E048F05FF68
:104C7600126FB78D068C07AC5AAD5BCFCECF120044
:104C860003740A8E048F05FF126FB78C5A8D5BAEC4
:104C960028AF29EF2DFDEE3CFC8C288D29024E42D3
:104CA6009000DBE0855FF0A4FFAEF07405126FC7DD
:104CB60074071200398E5A8F5B90009AE0A852B89A
:104CC60000049553501290009BE075F002A4FDACD1
:104CD600F0EFC39DEE9C4003024E42E55F75F00B7C
:104CE60084FF7E00900618120048FEE0FFEE90005A
:104CF60092E0FEEF8E0088F0A4FFAEF074648E049E
:104D06008F05FF126FB78C5A8D5B90005CE075F0D3
:104D160018A4FFAEF09000D9E08E048F05FF126F45
:104D2600B78C068D07900630120048AE5AAF5BE08E
:104D3600126FC774648E048F05FF126FB78C5A8D7D
:104D46005BE565A85AB80077D3955B4072E565C305
:104D5600955BFFE4955AFE8E5A8F5B7428BE00035E
:104D66009F500C755B28755A00740D90005DF0AE6F
:104D76005AAF5B900093E0126FC774288E048F05BC
:104D8600FF126FB78C5A8D5BAE28AF29740A8E045A
:104D96008F05FF126FB78D068C07AC5AAD5BCFCE71
:104DA600CF120003740A8E048F05FF126FB78C5A58
:104DB6008D5BAE28AF291270128E288F29807DE573
:104DC60065A85AB80004955B5072AE5AAF5BE565AC
:104DD60012700A8E5A8F5B7428BE00039F500C75A2
:104DE6005B28755A00740D90005DF0AE5AAF5B906B
:104DF6000093E0126FC774288E048F05FF126FB7F9
:104E06008C5A8D5BAE28AF29740A8E048F05FF126B
:104E16006FB78D068C07AC5AAD5BCFCECF120003B1
:104E2600740A8E048F05FF126FB78C5A8D5BAE28FD
:104E3600AF29EF2DFDEE3CFC8C288D29229000EE4B
:104E4600E0B4026AE55F75F00884FF7E008F37E5FF
:104E56005F75F00884ADF07C008D3A753F08755A91
:104E660001755BE0E537C3943F5005124287800623
:104E7600900287E0F53785372D752C00AE2CAF2DC7
:104E8600AC2AAD2B12000374648E048F05FF126FDB
:104E9600B78C2C8D2D90008BE08C068D07126FC77A
:104EA60074648E048F05FF126FB78C2C8D2DAE287F
:104EB600AF29AC2AAD2B12000374648E048F05FF54
:104EC600126FB78C288D2990008BE08C068D071207
:104ED6006FC774648E048F05FF126FB78C288D29F7
:104EE600A203401DAE52AF537405BE00039F50028D
:104EF600D203E561D394CC4008D201741190005DD1
:104F0600F09000EDE0B402089000DBE0640B600274
:104F16008035AE28AF29E56B126FC774E78E048F14
:104F260005FF126FB78C288D299000EEE0B40217AA
:104F3600AE2CAF2DE56B126FC774E78E048F05FF9D
:104F4600126FB78C2C8D2D9000ADE05402601B9033
:104F560000A4E0A852B80012D39553400DA203B3A3
:104F6600B35007E561C3949A40028028AE34AF354A
:104F76009000A2E075F002A4FDACF0EF2DFDEE3C32
:104F8600FC74022DFD50010CE561BC0007D39D4069
:104F960003754301856135753400E543700302509E
:104FA60086900100E0C395435003025078900110AB
:104FB600E0C394025076E56775F00A84FF7E0090A0
:104FC6000588120048E0F55B755A00AE5AAF5B9053
:104FD60000A3E0126FC774648E048F05FF126FB7CB
:104FE6008C5C8D5D900100E004C395438C068D07B3
:104FF600126FC7900100E08E048F05FF126FB78C09
:105006005C8D5DAE28AF29EF2DFDEE3CFC8C288D26
:10501600299000EEE0B40212AE2CAF2DAA5CAB5D77
:10502600EF2BFBEE3AFA8A2C8B2D8046900100E09E
:1050360004C39543854BF0A4FFAEF0900100E08ECB
:10504600048F05FF126FB78C5C8D5DAE28AF29EF1C
:105056002DFDEE3CFC8C288D299000EEE0B402126A
:10506600AE2CAF2DAA5CAB5DEF2BFBEE3AFA8A2C89
:105076008B2D0543900100E0C39543500375430013
:105086009000ADE05401601B9000A1E0A852B8006A
:1050960012D39553400DA203B3B35007E55FC394F3
:1050A600CC4002802590009FE075F003A4FFAEF08F
:1050B600E5402FFF50010E74032FFF50010EE55FF0
:1050C600BE0007D39F4003754401855F40E54470E9
:1050D600030251B9900101E0C3954450030251AB5C
:1050E600900110E0C394025076E56775F00A84FFDC
:1050F6007E00900588120048E0F55B755A00AE5AAE
:10510600AF5B9000A0E0126FC774648E048F05FF3A
:10511600126FB78C5C8D5D900101E004C395448CE1
:10512600068D07126FC7900101E08E048F05FF12EE
:105136006FB78C5C8D5DAE28AF29EF2DFDEE3CFC84
:105146008C288D299000EEE0B40212AE2CAF2DAA69
:105156005CAB5DEF2BFBEE3AFA8A2C8B2D804690EA
:105166000101E004C39544854CF0A4FFAEF0900124
:1051760001E08E048F05FF126FB78C5C8D5DAE2843
:10518600AF29EF2DFDEE3CFC8C288D299000EEE03A
:10519600B40212AE2CAF2DAA5CAB5DEF2BFBEE3A40
:1051A600FA8A2C8B2D0544900101E0C395445003E7
:1051B600754400900103E02529FFAE2850010E8EAC
:1051C600288F299000B2E0A828B800049529500934
:1051D6009000B2E0F5297528009000EEE0B4020DCB
:1051E6009000B2E0A82CB80006952D4002800990E8
:1051F60000B2E0F52D752C00229000EEE0B401021D
:10520600800302530AA203B350030253089000B965
:10521600E0B40168AE28AF29AC52AD531200037456
:105226003C8E048F05FF126FB79000C9E0BC0010DA
:105236009D400D9000CBE0A828B8000495295002A7
:10524600D202AE28AF29AC52AD53120003743C8E85
:10525600048F05FF126FB79000C9E0C3940ABC0023
:1052660015D39D40119000CBE0C39405A828B80043
:1052760005D3952950028002C2028068AE28AF2964
:10528600AC52AD5312000374788E048F05FF126F73
:10529600B79000C9E0BC00109D400D9000CBE0A87F
:1052A60028B8000495295004D2028038AE28AF29C8
:1052B600AC52AD5312000374788E048F05FF126F43
:1052C600B79000C9E0C3940ABC0015D39D40119065
:1052D60000CBE0C39405A828B80005D39529500251
:1052E6008002C202A202B34019AE28AF299000CABA
:1052F600E0126FC774648E048F05FF126FB78C2897
:105306008D298002C202A200B34006A201B3B350A7
:105316000990001FE4F0A3F08024AE28AF297400A2
:10532600D39F74019E400C90001FE528F0A3E52949
:10533600F0800B74FF90001FF8E4F0E8A3F09000F3
:10534600B9E0B4011AAE28AF297402126FC78E28CD
:105356008F29AE2CAF2D7402126FC78E2C8F2D9015
:1053660000D0E0C394034009900084E0C394025047
:1053760035AE28AF29745E126FC7740A8E048F0586
:10538600FF126FB78C288D299000EEE0B40217AE9D
:105396002CAF2D745E126FC7740A8E048F05FF1230
:1053A6006FB78C2C8D2DAE28AF297402BE000AD3A0
:1053B6009F4006752902752800AE2CAF2D7402BEDB
:1053C600000AD39F4006752D02752C0090001DE53E
:1053D60028F0A3E529F02290005CE0900388126F84
:1053E600F8E0F54175426490005CE0FE9000C4E090
:1053F600D39E4037E55F75F00884FF7E008F37E562
:105406005F75F00884ADF07C008D3A753F08755ADB
:1054160003755B96E537C3941F50051242878006D5
:1054260090043DE0F5378537428035E55F75F00835
:1054360084FF7E008F37E55F75F00884ADF07C0051
:105446008D3A753F08755A03755BB6E537C3941FE9
:105456005005124287800690045DE0F53785374295
:10546600229000FAE0F53C753F11755A04755B0011
:10547600AE52AF53E53C75F00FA4FDACF0EDD39FF3
:10548600EC9E4021E53C8E048F05FF126FB7ED754B
:10549600F010A4FFAEF0E55F75F01184FD7C00ED21
:1054A6002FF53D800EE55F75F01184FF7E00EF2439
:1054B600F0F53D853D37E55F75F01184AFF07E0070
:1054C6008F3A12428785373EAE52AF539000FAE0CC
:1054D60075F00FA4FDACF0EDD39FEC9E4028755AF5
:1054E60004755B10853D37124287853E388537390E
:1054F600AE52AF53E53C8E048F05FF126FE28D3A34
:10550600853C3B124301853741754264229000FA7F
:10551600E0F53C753F11755A04755B00AE52AF530A
:10552600E53C75F00FA4FDACF0EDD39FEC9E402159
:10553600E53C8E048F05FF126FB7ED75F010A4FFE2
:10554600AEF0E56175F01184FD7C00ED2FF53D8030
:105556000EE56175F01184FF7E00EF24F0F53D85C0
:105566003D37E56175F01184AFF07E008F3A124247
:105576008785373EAE52AF539000FAE075F00FA420
:10558600FDACF0EDD39FEC9E4028755A04755B1078
:10559600853D37124287853E38853739AE52AF533F
:1055A600E53C8E048F05FF126FE28D3A853C3B1277
:1055B60043018537417542649000F5E0B404799063
:1055C600005CE0FE9000C4E0D39E4037E55F75F0D6
:1055D6000884FF7E008F37E55F75F00884ADF07CA8
:1055E600008D3A753F08755A03755B96E537C39487
:1055F6001F5005124287800690043DE0F537853737
:10560600428035E55F75F00884FF7E008F37E55FE1
:1056160075F00884ADF07C008D3A753F08755A0325
:10562600755BB6E537C3941F500512428780069016
:10563600045DE0F5378537422290008EE0B4013BE9
:10564600E56775F00A84FF7E008F37E56775F00A17
:1056560084ADF07C008D3A753F0A755A05755B126C
:10566600E537C39411500512428780069005ABE0DA
:10567600F537E5422537C39464F54290008FE0B4D0
:10568600013BE56875F00A84FF7E008F37E5687593
:10569600F00A84ADF07C008D3A753F0A755A05759F
:1056A6005B7EE537C394115005124287800690064B
:1056B60017E0F537E5422537C39464F542E5412501
:1056C60042F536900096E0B402109008B4E0253614
:1056D600FE9000EAE0F4042EF5369000EDE0D39457
:1056E600014040E56BC394E7501D74E7C3956BFE1C
:1056F6009008B6E08E00F5F0E884FF7E008F37E56F
:10570600362537F536801CE56BC394E7FE9008B660
:10571600E08E00F5F0E884FF7E008F37E536C3950E
:1057260037F536A2034006E5412464F536E536D35F
:1057360094644009E536C39464F5368003753600F3
:105746009000C6E0C3953650069000C6E0F53622B6
:10575600D200900078E0A852B800049553503E90CD
:105766000078E0A852B800049553500375360F90A0
:105776000078E004A852B800049553500375360724
:10578600900078E02402A852B8000495535002C253
:1057960000900078E06006740990005DF0C2307EEB
:1057A600017F009000CCE0126FC79000DBE08E0412
:1057B6008F05FF126FB7E55FBC0017D39D401390AE
:1057C60000D5E0B40204D2308002C200740A900010
:1057D6005DF090008EE0B401099000CDE0C39567BE
:1057E600400280159000DFE0A852B800049553509F
:1057F60002C200740B90005DF090008EE0B40107C9
:10580600E567C394644002801D900125E0600D9019
:105816000125E0A852B80006955340028008C20050
:10582600740B90005DF0A200400375360090010EE7
:10583600E0B4011490010FE0A852B800049553504B
:1058460007E55FC39560400280209000B7E0D394DF
:105856001D400B9000B7E0C3941EF53680037536E5
:1058660000741590005DF0025947900096E0B4036D
:1058760006A229B3B340030259479008B8E0C3947F
:1058860005A852B80004955350069008BEE0600281
:10589600801D9000B7E0D3941D400B9000B7E0C385
:1058A600941EF5368003753600740C90005DF090FA
:1058B60008B8E0A852B80004955350069008BEE018
:1058C6007002801D9000B7E0D3941D400B9000B786
:1058D600E0C3941EF5368003753600740C90005DA7
:1058E600F09008B8E0A852B80004955350319000E3
:1058F600D5E0B40228D2309008BDE0FE9008BEE0A4
:10590600D39E50069008BEE0700280099008BDE460
:10591600F0C23080069008BDE004F08002C200901C
:1059260008B8E02405A852B8000495535013900017
:10593600D5E0B4020A9008BEE07002D2308002C2FE
:1059460000A22FB3401D9000B7E0D3941D400B90EA
:1059560000B7E0C3941EF5368003753600741090C8
:10596600005DF085366C9000B7E0D3941D4018902A
:105976000085E02536FE90005CE075F01E84FC7F15
:1059860000EE2CF536804990005DE0640C600F90C7
:10599600005DE06410600790005DE0B415169000AD
:1059A60085E0FE90005CE075F01E84FC7F00EE2C26
:1059B600F536801C900087E02536FE900085E02EA7
:1059C600FE90005CE075F01E84FC7F00EE2CF53640
:1059D6002290005CE075F00584FF7E008F37900012
:1059E6005CE075F00584ADF07C008D3A753F057579
:1059F6005A03755BD69000D9E01475F00584FF7ED6
:105A060000E537BE00039F5005124287800BE5373D
:105A160090045E126FF8E0F537E5379008B7F0901E
:105A260008B7E0FE9000C8E0C39E50089000C8E0AA
:105A36009008B7F022E56775F00A84FF7E009005AE
:105A460088120048E0F546E546D394644010E546E2
:105A5600C3946475F00F84FF7E008F4680037546FD
:105A6600009000ABE02546F54622E56775F00A840E
:105A7600FF7E00900588120048E0C3946950559057
:105A860000F5E0C39403502690088AE0FEA3E0FFE9
:105A96007404120039E55F126FC7740F8E048F0508
:105AA600FF126FB7900888ECF0A3EDF08024900801
:105AB6008AE0FEA3E0FF7404120039E561126FC7A5
:105AC600740F8E048F05FF126FB7900888ECF0A351
:105AD600EDF0800F90088AE0F8A3E0900888C8F0FF
:105AE600A3C8F0A203401A90088AE0FEA3E0FF7460
:105AF60003126FC77401120039900888EEF0A3EF05
:105B0600F0900888E0FEA3E0FF90088EE0FCA3E09A
:105B1600FDEDD39FEC9E400F90088EE0F8A3E09039
:105B26000888C8F0A3C8F090009EE0B40262E56A57
:105B3600C3944175F00584FF7E008F37E56A75F0E2
:105B46000584ADF07C008D3A753F05755A06755B88
:105B560014E537C39417500512428780069006AFA6
:105B6600E0F537900888E0FEA3E0FF740A8E048F04
:105B760005FF126FB7E5378C068D07126FC7740ADB
:105B86008E048F05FF126FB7900888ECF0A3EDF036
:105B960022E50875F004A4FFAEF09006CB1200488B
:105BA600E09068CBF8282873804C85537380479023
:105BB60000DBE0855FF0A4FFAEF074081200398FB9
:105BC600738033856173802E85677380298568733A
:105BD6008024856973801F856A73801A856B73803C
:105BE600158566738010856573800B856C738006DA
:065BF600900020E0F573B1
:1068CB00025BAE025BB0025BB5025BC9025BCE0240
:1068DB005BD3025BD8025BDD025BE2025BE7025B30
:0768EB00EC025BF1025BF619
:105BFC00E50875F004A4FFAEF09006CC120048E561
:105C0C000875F004A4FFAEF0E0FC9006CD1200483D
:105C1C00ECFEE0FFEEC39F4003025D04E50875F067
:105C2C0004A4FFAEF09006CB120048E0B40441E5AA
:105C3C000875F004A4FFAEF09006CD120048E0C346
:105C4C009573500AE508F50CD39231120EC8E5088D
:105C5C0075F004A4FFAEF09006CC120048E0D3958A
:105C6C0073400AE508F50CC39231120EC8025D02AE
:105C7C00E50875F004A4FFAEF09006CC120048E0E5
:105C8C00C395735015E50875F004A4FFAEF09006AB
:105C9C00CD120048E0D395735002800AE508F50C4C
:105CAC00D39231120EC8E50875F004A4FFAEF09043
:105CBC0006CC120048E0D395735015E50875F00436
:105CCC00A4FFAEF09006CD120048E0C39573500AC5
:105CDC00E508F50CC39231120EC89006D3E0B4015E
:105CEC00099000E7E0D395615002800A7402F50C2C
:105CFC00C39231120EC8806AE50875F004A4FFAE99
:105D0C00F09006CC120048E0D395734015E5087569
:105D1C00F004A4FFAEF09006CD120048E0C39573DA
:105D2C004002800AE508F50CC39231120EC8E50852
:105D3C0075F004A4FFAEF09006CC120048E0C395B9
:105D4C00734015E50875F004A4FFAEF09006CD1273
:105D5C000048E0D39573400AE508F50CD392311254
:105D6C000EC822AE2EAF2F74C9BE000CD39F4008B4
:105D7C00782E12701A025E89752F01752E00AE52A4
:105D8C00AF53E546BE000DD39F40099000BDE0D354
:105D9C00954740028023754700E546C39553F5733C
:105DAC009000C0E0D395454008E5452573F5458046
:105DBC00069000C0E0F54580020547900099E0D3BD
:105DCC009561401CE55FC395604015AE52AF53E53D
:105DDC0046BE00039F50099000BEE0D39548400298
:105DEC00806E9008B9E0A852B80004955350037522
:105DFC004A009008B9E0A852B8000BD3955340065E
:105E0C00E5539008B9F0E54A7041E553C39546F562
:105E1C0073E573D3940540037573059000BFE0C31D
:105E2C0095455007E573C3954540028009E545C388
:105E3C009573F54580069000BFE0F5459000BFE0F6
:105E4C00D3954540069000BFE0F5457548008002AB
:105E5C000548E54A7016900099E0C39561500DE530
:105E6C00462405A852B8000695534002800F9000B6
:105E7C00ACE0F545754A0174789008B9F022AE2E65
:105E8C00AF2F74E9D39F74039E4008782E12701ABA
:105E9C00026030752F01752E00754532A22A402AFA
:105EAC007545199000ACE075F002A4FFAEF0E54723
:105EBC00BE0006D39F4002D22A0547754A03747868
:105ECC009008B9F0754900026017AE52AF53E54621
:105EDC006F4E7003026017E546BE000DD39F40095C
:105EEC009000BDE0D395474002800F754700E54A0E
:105EFC00C394035003754519800DE546C39553F5BE
:105F0C0073E5472573F547900099E0D39561400EF2
:105F1C009008B9E0A852B80007D395534002800C02
:105F2C0005499000ACE0B54903754A00E54AB40355
:105F3C0006A203B3B34002800A0549E549B43C0309
:105F4C00754A02E54AB402299008B9E0A852B80093
:105F5C000ED395534009E5539008B9F0754900905C
:105F6C000099E0C39561500975490074789008B99F
:105F7C00F0E54A705A900099E0D39561401CE55FBA
:105F8C00C395604015AE52AF53E546BE00039F501B
:105F9C00099000BEE0D39548400280087548007512
:105FAC00454B8028E553C39546F573E573D39405AB
:105FBC004003757305900099E0D395614008E5485E
:105FCC002573F5488006E5482406F548754900E533
:105FDC004A7016900099E0C39561500DE546240572
:105FEC00A852B80006955340028003754A01E54A51
:105FFC00B4011875451905499000ACE0B549067512
:10600C004A0275490074789008B9F0A201B34003B4
:10601C00754532E54575F00AA4FFAEF0900890EE98
:10602C00F0A3EFF022E56F9068F2F8282873900047
:10603C0091E0700302626E9000C7E0B4010280032D
:10604C0002617990005AE0655E6009E55345526043
:10605C00030261767E017F00E5BE126FC7E5BD2F9E
:10606C00FF50010E8E5A8F5B7410126FC790007721
:10607C00E08E048F05FF126FB7900894ECF0A3ED3F
:10608C00F0E56B600FE56BC394FE50089000EDE0FB
:10609C006402600280649000DBE0B40B1F900894F3
:1060AC00E0FEA3E0FF74E7126FC7E56B8E048F056B
:1060BC00FF126FB7900894ECF0A3EDF09000DBE0CA
:1060CC00D3940B40089000C3E064046002802B90D2
:1060DC000894E0FEA3E0FF900898E0FCA3E0FDEF3D
:1060EC00D39DEE9C400D127012900894EEF0A3EF2D
:1060FC00F08007900894E4F0A3F0900091E0B402D3
:10610C0027900896E0FEA3E0FF900894E0FCA3E043
:10611C00FDEF2DFDEE3CFC74018C068D0712003951
:10612C00900894EEF0A3EFF0900894E0FEA3E0FF4B
:10613C00900896E0FCA3E0FDEDD39FEC9E4004D2CA
:10614C002E8002B22E900894E0F8A3E0900896C836
:10615C00F0A3C8F09000C3E064016006A22EB3B3B4
:10616C0040028006900895E0F55F02626CD22E7EAC
:10617C00017F00E5BE126FC7E5BD2FFF50010E8EEB
:10618C005A8F5B7410126FC7900077E08E048F05E6
:10619C00FF126FB7900894ECF0A3EDF0E56B600F75
:1061AC00E56BC394FE50089000EDE0640260028041
:1061BC00649000DBE0B40B1F900894E0FEA3E0FFBA
:1061CC0074E7126FC7E56B8E048F05FF126FB790E3
:1061DC000894ECF0A3EDF09000DBE0D3940B4008B6
:1061EC009000C3E064046002802B900894E0FEA34E
:1061FC00E0FF900898E0FCA3E0FDEFD39DEE9C40FF
:10620C000D127012900894EEF0A3EFF08007900836
:10621C0094E4F0A3F0900091E0B40227900896E08B
:10622C00FEA3E0FF900894E0FCA3E0FDEF2DFDEE53
:10623C003CFC74018C068D07120039900894EEF02A
:10624C00A3EFF0900894E0F8A3E0900896C8F0A3B0
:10625C00C8F09000C3E064016006900895E0F55F1B
:10626C008003755F0090008DE07006756F01026011
:10627C003175BB180268A590008DE070030263F4C1
:10628C007E017F00E5BE126FC7E5BD2FFF50010EEA
:10629C008E5A8F5B9000D3E0B4010F7E0F7FFFAC62
:1062AC005AAD5B1270128E5A8F5B9000F8E0B402FC
:1062BC0045AE5AAF5B900029E0FCA3E0FDEDD39F07
:1062CC00EC9E400A900029E55AF0A3E55BF0AE5A2B
:1062DC00AF5B90002BE0FCA3E0FDEFD39DEE9C4068
:1062EC000A90002BE55AF0A3E55BF0AE5AAF5B7455
:1062FC00041200398F619000F8E0704CAE5AAF5B1D
:10630C00900029E0FCA3E0FDEFD39DEE9C40091228
:10631C0070128E5A8F5B8006755B00755A00AE5AF0
:10632C00AF5B7410126FC7900074E08E048F05FF82
:10633C00126FB78C5A8D5B74FFBC0009D39D40055E
:10634C00855B6180037561FE9000C3E0B40102803F
:10635C00030263F2A203B3B3500E900097E0A8526D
:10636C00B80005D39553500280719000D4E085613C
:10637C00F0A4FFAEF074648E048F05FF126FB78C1F
:10638C005A8D5BE56B6016E56BC394FE500F900065
:10639C00EDE0B402089000DBE0640B60028017AE05
:1063AC005AAF5B74E7126FC7E56B8E048F05FF1253
:1063BC006FB78C5A8D5BAE5AAF5B900894E0FCA320
:1063CC00E0FDEDD39FEC9E4005855B5F800BA22E1C
:1063DC00B34006900895E0F55F800BA22EB3400603
:1063EC00900895E0F55F8003756100900090E07077
:1063FC0006756F0202603175BB190268A59000909A
:10640C00E070030264A9E55ED3955140030264A7D2
:10641C00900027E0FEA3E0FFE56512700A900027CC
:10642C00EEF0A3EFF07E017F00E5BE126FC7E5BD75
:10643C002FFF50010E8E5A8F5B9000FDE07013748D
:10644C000A126FC774518E048F05FF126FB78D65DA
:10645C008019AE5AAF5B740A126FC78F048E057E1B
:10646C00017F95CDCCCD126EB58F65E565D3946467
:10647C004003756564900027E0FEA3E0FFE5652FFF
:10648C00FF50010E900027EEF0A3EFF0900094E087
:10649C00048E048F05FF126FB78D6580037565320E
:1064AC009000E0E07006756F0302603175BB13025B
:1064BC0068A59000E0E0604A7E017F00E5BE126FA7
:1064CC00C7E5BD2FFF50010E8E5A8F5B740412006E
:1064DC00398F669000E2E08566F0A4FDACF0746440
:1064EC00FF126FB78D669000E1E08566F0A4FFAEF9
:1064FC00F074FF8E048F05FF126FB7ED900073F0F0
:10650C00800375660090008EE07006756F04026063
:10651C003175BB170268A590008EE0B401028003B0
:10652C000265B77E017F00E5BE126FC7E5BD2FFF88
:10653C0050010E8E5A8F5B9008BAE060199008BA21
:10654C00E0149069C212008CE493FC740193FDED8D
:10655C00C39FEC9E400280069008BAE014F09008AD
:10656C00BAE0C394B3501DAE5AAF5B9008BAE004C6
:10657C009069C212008CE493FC740193FDEFC39DEF
:10658C00EE9C400280069008BAE004F09008BAE055
:10659C00FE9000B4E08E0088F0A4FFAEF074648E20
:1065AC00048F05FF126FB78D67800375670090002D
:1065BC008FE07006756F0502603175BB160268A519
:1065CC0090008FE0B4010280030266607E017F00C0
:1065DC00E5BE126FC7E5BD2FFF50010E8E5A8F5BC3
:1065EC009008BBE060199008BBE014906B2C120073
:1065FC008CE493FC740193FDEDC39FEC9E400280F0
:10660C00069008BBE014F09008BBE0C394B3501D97
:10661C00AE5AAF5B9008BBE004906B2C12008CE47C
:10662C0093FC740193FDEFC39DEE9C400280069099
:10663C0008BBE004F09008BBE0FE9000BAE08E00CE
:10664C0088F0A4FFAEF074648E048F05FF126FB750
:10665C008D68800375680075BB1F0268A57E017F7D
:10666C0000E5BE126FC7E5BD2FFF50010E8E5A8F8D
:10667C005B7409126FC774E68E048F05FF126FB737
:10668C008D6A900096E07006756F0702603175BBDD
:10669C00150268A5900096E070030267F17E017FF9
:1066AC0000E5BE126FC7E5BD2FFF50010E8E5A8F4D
:1066BC005B74041200398F69900096E0B401159058
:1066CC0000EAE08569F0A4FFAEF07407120039EF20
:1066DC009008B5F0900096E0B402159000EAE085C1
:1066EC0069F0A4FFAEF07407120039EF9008B4F013
:1066FC00900096E0B4030280030267D49000D7E0C8
:10670C007052E569C39419500FD2299000B6E090ED
:10671C0008B8F09008BCE4F0E569D394644004A296
:10672C00294002802D9008BCE004F09008BCE0FEEB
:10673C00900129E0B5060B9008B8E004F09008BC75
:10674C00E4F09008B8E064966006900129E07002CD
:10675C00C22980639000B6E070349000EAE085694D
:10676C00F0A4FFAEF074FF8E048F05FF126FB7ED2F
:10677C009008B8F0AE52AF53741EBE0006D39F40C3
:10678C0002D229E561D394E54002C2298029E5694A
:10679C00C3940A500DAE52AF53741EBE0004D39F67
:1067AC0050028002D229E561D394E54002C22990BF
:1067BC0000B6E09008B8F09008B8E0C39405500615
:1067CC0074059008B8F0C22F900096E0B40414E55C
:1067DC0069C394195002D22FE569D394324002C296
:1067EC002FC22980037569009000EDE07006756F6B
:1067FC000802603175BB140268A59000EDE07003CF
:10680C000268947E017F00E5BE126FC7E5BD2FFFC5
:10681C0050010E8E5A8F5B900112E07025EFD394CD
:10682C0021EE940E4005756BFF8015AE5AAF5B746C
:10683C0010126FC774E38E048F05FF126FB78D6B48
:10684C008027AE5AAF5BEFD39449EE9406400575A2
:10685C006BFF8015AE5AAF5B7410126FC774658EE8
:10686C00048F05FF126FB78D6BE56B75F00BA4FFF2
:10687C00AEF09000DBE08E048F05FF126FB790082E
:10688C0098ECF0A3EDF08003756B00900091E06044
:09689C000575BB1A800375BB18D9
:1068F20002603A0262830264090264BE02652302F4
:0B69020065CC0266690266A002680610
:0568A500056FD2EC229A
:096FF8002582F582500205832276
:0F008C0025E050020583258250020583F582226C
:106F9600EF2F500205832582F582E5833E2EF58389
:016FA60022C8
:10700A00CFC39FFF50011E22C3EF9DFFEE9CFE22BD
:08701A000806B6000218062268
:0D6FD500A3E004F07006126FEEE004F0225D
:0E003900048007C3CE13CECF13CFD5E0F6223E
:106EB500BC000FBE0008ED8FF084FFADF022E4FEAC
:106EC500FF22BE000DEF60FE54F0606F20E7030265
:106ED5006F6BEAC0E0EBC0E078017A0075F001EE77
:106EE50020E710EF25E0FFEE33FE0AC5F023C5F0DD
:106EF50030E7F0EA5407F9096A7A007B0060010877
:106F0500C3EC9E40167004ED9F4010ED9FFDEC9E76
:106F1500FCE5F0CA4ACA03F5F08005E5F003F5F093
:106F2500C3EE13FEEF13FFD9D77908CACBCAD8D061
:106F3500EAFEEBFFD0E0FBD0E0FA22EC8FF084FC18
:106F4500ED54F045F0C48FF084FEEDC454F045F0E7
:106F5500C48FF084FDEEC4FE54F02DFFEE540F3CBB
:106F6500FEADF07C0022790078008FF0EC7E0820E1
:106F7500E70DC3CD33CD33C933C9C833C8DEF0847B
:106F850049F9E5F08FF0BE00E6FD7C00E9FFE8FE7B
:016F950022D9
:0E6FC700F88FF0A4FFE5F0CE88F0A42EFE2295
:10000300EF8DF0A4F9A8F0EF8CF0A428F8EE8DF0B2
:06001300A428FEE9FF2213
:106FA700600D782B026FB1007830D8FED5E0F8225B
:106FB700EEC0E07E00126EB5EFFDEEFCD0E0FE22E3
:0C6FE200EEC0E07E00126EB5D0E0FE2292
:03001B0002001EC2
:0300530002005652
:03009B00020071EF
:030000000270018A
:0970010075817575D00002117350
:0B004800E5822FF582E5833EF5832260
:0A6FEE000582D58202158315822268
:10001E00C0E0C0F0C083C082C0D075D0001210798D
:0B002E00D0D0D082D083D0F0D0E032E0
:10005600C0E0C0F0C083C082C0D075D00012107C52
:10006600D0D0D082D083D0F0D0E032C0E0C0F0C093
:1000760083C082C0D075D000121126D0D0D082D0D5
:0600860083D0F0D0E0324F
:00000001FF
